:020000020000FC
:0200000037C007
:02000800567828
:100034000C94132B0C94112B4156522D4368697068
:100044004261736963322028632920323030362DAF
:1000540032303038204A6F65726720576F6C667291
:04006400616D0000CA
:10007000F894A0E02A2EA1E03A2EA0E1AEBFAFEFA7
:10008000ADBFB0E0A0E0AA95F1F7BA95D9F70E940C
:10009000A32C0E94DA380E940E790E9472340E94CA
:1000A000FD2DAFEFA093310120923D0120923E0142
:1000B000209250018827789420922D01A091290147
:1000C000A4FD0C946A000E94FD2D0E94A2010E94D2
:1000D0005932CECFA1E00E94732DAA270E941D2D78
:1000E0009927A7E10E946E2D0E94FD2DA0E10E949C
:1000F0006E2DC4E0DAE0E7E3F7E10E944131A7E0CA
:100100000E946E2D0E94F22F070420008AD1A6E1E2
:100110000E946E2DC5E0D8E0E6E0F9E00E94413192
:10012000D8E1F9E10E944131D8E0F9E0CC5FEC5F21
:10013000C833A0F366E90E9430326A95E1F70C9467
:10014000A100A0E00E94732DA1E00E94E533992751
:1001500020922A01AA270E941D2DA5E10E946E2D42
:100160000E94FD2DC0E0D0E0EDE1F4E10E94953168
:10017000A1E50E946E2D0E94F22F010183838383EB
:100180008383204156522D436869704261736963CD
:1001900032208282828282820000A9E9B4E00AE4ED
:1001A0000D9304EC0D930CE80D9308E20D9302E619
:1001B0000D9306EA0D93509606EA0D9302E60D9311
:1001C00008E20D930CE80D9304EC0D930AE40D93F3
:1001D00032D240913D014B3008F0442740933D011D
:1001E000642F67FD66276B3008F06AE050E06F937C
:1001F0002BD16F9153955830D1F7F3D1C8D19DD100
:100200006F939CD26F91423E11F46A95EACF433EC0
:1002100011F46395E6CF443E21F4643010F064504D
:10022000E0CF453E21F4673010F46C5FDACF6830E0
:10023000F8F04A3E11F0443F19F760933D016830F1
:1002400039F44A3EE9F6FBD00E94B51BF8D079CFCD
:10025000693039F44A3EA1F6F2D00E946420EFD012
:1002600070CFEDD04A3E61F60E94F721E8D069CF09
:100270004F934091140142FD2AC04F914A3E11F024
:10028000443F41F460933D01DAD088270E94A201E7
:10029000D6D057CF413F41F460933D01D0D088275D
:1002A0000E948C01CCD04DCF423F39F460933D0188
:1002B000C6D00E94631DC3D044CF433F39F460933E
:1002C0003D01BDD00E94C81DBAD03BCF99CF4F9100
:1002D000413F39F460933D01B2D00E94B403AFD0E6
:1002E00030CF423F39F460933D01A9D00E948B2268
:1002F000A6D027CF433F39F460933D01A0D00E94A0
:10030000C6229DD01ECF443F09F760933D0197D090
:100310000E94FC0394D015CFA0911601A030E1F704
:100320000E94700420922D01A0911701A43F09F0B2
:1003300008CF08D00E946032A0E00E941D2D0E94CC
:10034000FD2DEACF0E94FD2D8827209216010E94E4
:100350000D7A3C9645914E3411F4339609940E94DF
:100360000E0E20920D012092500120922A010E942F
:10037000372EA7E20E946E2D92E0A0913E01A030A0
:1003800079F0A33021F4A7E20E946E2D09C0A0E10C
:100390000E946E2DA0E4A0930001A0EEA0930101A5
:1003A000A0913E01A03051F40E94F22F160020507F
:1003B000524553532045534320002EC0A13051F4E1
:1003C0000E94F22F69002050524553532045534359
:1003D000200022C0A23051F40E94F22F420020508F
:1003E0005245535320455343200016C0A33049F4CF
:1003F0000E94F22F2F002050524553532045534363
:100400002000A53049F40E94F22F380020505245B8
:100410005353204553432000A0911601AD3EE1F710
:1004200008950E94F22FFF4156522D436869704291
:1004300061736963322056302E3836000895A091DA
:100440001601A030E1F70895A1E0B3E050FDA95FE7
:1004500051FDA25F52FDBA5F4EE2651709F4429565
:1004600040932C010E940B300E94F22FFF202000AD
:1004700040E50E94642E452F4F5C0E94642E0E942E
:10048000F22FFF202000B3950E940B30452F0E94D1
:100490000F7A3C9645914E3481F40E94F22FFF2052
:1004A00020E6E7202000B3950E940B300E94F22F37
:1004B000FF2020E8E920200021C0423481F40E947E
:1004C000F22FFF2020D0D1202000B3950E940B30C6
:1004D0000E94F22FFF2020D2D32020000FC00E94C4
:1004E000F22FFF2020CACB202000B3950E940B30B2
:1004F0000E94F22FFF2020CCCD202000452F0E940B
:100500000F7AB3950E940B3066E045910E94642EED
:100510006A95D9F7B3950E940B3066E045910E9429
:10052000642E6A95D9F7B3950E940B300E94F22F82
:10053000FF2020202020200008954AE26A3009F49C
:10054000429540932C010E94F22F0F0F2020202073
:10055000202000000E94F22F100F2020D4D5202050
:1005600000000E94F22F110F2020D6D7202000007B
:100570000E94F22F120F20494E464F2000000E9489
:10058000F22F130F2020202020200000089548E2A1
:10059000693009F4429540932C010E94F22F0F0814
:1005A00020202020202000000E94F22F1008202070
:1005B000D8D9202000000E94F22F11082020DADB79
:1005C000202000000E94F22F1208434F4E46494758
:1005D00000000E94F22F130820202020202000007D
:1005E00008954CE2683009F4429540932C010E9432
:1005F000F22F0F0120202020202000000E94F22F47
:1006000010012020DCDD202000000E94F22F1101CB
:100610002020DEDF202000000E94F22F120144463D
:100620004C41534800000E94F22F1301202020204B
:10063000202000000895A0E00E946E2D0E94F22F5D
:1006400015002020202020202020202020202020D5
:10065000202020202020202020202020202020209A
:100660000000A7E20E946E2D0E94F22F16002020AB
:10067000202020200000A0E60E946E2D0E94F22F74
:1006800016062045646974200000A0E40E946E2DC7
:100690000E94F22F160C2053617665200000A7E11E
:1006A0000E946E2D0E94F22F1612204C6F61642062
:1006B0000000AEE6A0932B07A7E30E946E2D0E94D8
:1006C000F22F16182052756E20000895A0E00E94A7
:1006D0006E2DA7E20E946E2D0E94F22F16002020A0
:1006E000202020200000A0E60E946E2D0E94F22F04
:1006F000160620436F7079200000A0E40E946E2D42
:100700000E94F22F160C2053656E64200000A7E1B2
:100710000E946E2D0E94F22F1612205265637620E1
:100720000000AEE6A0932B07A7E30E946E2D0E9467
:10073000F22F1618436C6561720008953DED20920A
:1007400017010E94FD32409114014470431739F0A3
:10075000342F403011F46FDFF4CFB8DFF2CF409187
:100760001701403071F30895A4E00E946E2DC1E09E
:10077000DFE0ECE1F3E10E949531A0E40E946E2DF0
:100780000E94F22F1002436F70792050726F6772CF
:10079000616D20746F0070913D0160E0ACE06717FF
:1007A00009F4A0E60E946E2DB2E1A62FAA0FA60FB3
:1007B000AD5F0E940B3040E50E94642E462F4770CB
:1007C0004F5C0E94642E6395683041F70E94593255
:1007D000423E21F47030D1F37A95DFCF433E21F4CD
:1007E0007730A1F37395D9CF4A3E19F40E94427A2B
:1007F00008954D3E59F708950E94CF364F436C65DA
:10080000617220746869732050726F6772616D3F06
:100810002000413009F008950E941C7A0895AA270B
:100820000E94732DA3E00E94E5338F9340913D0118
:100830000E9415790E94FD2D0E94122D992740914A
:1008400016014030E1F70E94F22F00002050524F75
:100850004752414D200040913D014F5C0E94642E63
:100860004AE30E94642EC3EDD1E059D2F1D20E9436
:10087000DC7904D48F91A8E8803069F1ACECE6EB28
:10088000F0E1813031F0ABE48A9545914030E9F7F1
:10089000F8CF4DD292E0A5E0B1E00E940B300E946B
:1008A000EA2F0E94F22FFF20494E20500000409175
:1008B0003A014F5C0E94642E4AE30E94642EBB27DB
:1008C000AC2DA3950E948D2D4AE30E94642EAD2D80
:1008D000A3950E948D2D0895AAE25A2E70E20895E4
:1008E0009927FADF9CDFD22CAA27BB27D0922E01B2
:1008F0000E9483320E94FD32403E11F4AA27F6CFB7
:10090000413E11F4AFE12BC0423E11F4AA9527C03D
:10091000433E69F4A3959B2F0E9494099A1730F4E3
:10092000BE3511F4AA951BC0AA27B39518C0443E42
:1009300021F4BA95B7FDBB2712C0463E21F4B8504A
:10094000B7FDBB270CC0473E11F4B85F08C0453E59
:1009500011F4B39504C04A3E39F5B395AA27A038DF
:1009600038F0AFE1BA95B038C0F0AA27BB27BECFA8
:10097000A03228F0BE3589F0AA27B395B7CFBF358E
:1009800008F0BEE50B2F0D1508F4D02E0D2D015FDC
:100990000B1718F40B2F0F50D02E9B2F0E94940989
:1009A0009A1708F4A92FA2CF9B2F4E3E39F4AF938C
:1009B000BF930E945609BF91AF918AC14F3E39F44F
:1009C000AF93BF930E946109BF91AF9181C1493E2E
:1009D00011F482D17DC14C3E31F4A03009F488CFAE
:1009E000AA957AD175C150911401547009F4C5C00B
:1009F000433FD1F4ACEC9BD10E94F22F010752454A
:100A000043454956452050524F4752414D20592F9A
:100A10004E203F006DD12EF48DD230D35DDF509249
:100A2000C8017DD1882760CF423F39F5ACEC7FD13A
:100A30000E94F22F010753454E442050524F475217
:100A4000414D20592F4E203F000052D156F7ACECBB
:100A50006ED10E94F22F010753454E44494E472E56
:100A60002E2E2020202020202020000030922A013D
:100A700093D120922A0130DFD4CF443FB1F4ACECC3
:100A800056D10E94F22F0107434C4541522050524B
:100A90004F4752414D20592F4E203F0029D126F477
:100AA000DBD21ADF5092C801BCCF413F41F5ACEC1C
:100AB0003ED10E94F22F01075052494E542050520D
:100AC0004F4752414D20592F4E203F0011D1B6F4CF
:100AD000ABE42DD10E94F22F01075052494E5449E8
:100AE0004E472E2E2E202020202020202000A2E065
:100AF000A0932A0151D120922A01EEDE92CF4336F3
:100B000071F462E46093E50165E56093E60166E4F3
:100B10006093E7016DE36093E80179D2E9CE48374D
:100B200091F462E46093E50165E56093E60166E4B3
:100B30006093E7016DE36093E8010E9407087CD2AF
:100B40005092C80118C04637B1F46091E501623493
:100B500099F460E26093E5016093E6016093E70138
:100B60006093E8016093E9016093EA0143D286D281
:100B70005092C801BDCE8827BBCE423F11F5BF932E
:100B8000AF93C9D0D9F0ACECD2D00E94F22F0107BC
:100B9000534156452050524F4752414D20592F4EF8
:100BA000203F0000A5D046F40E94A8790E94DC797D
:100BB00065D292DE7093C801B2D08827AF91BF9101
:100BC00095CE433FE1F4BF93AF93A5D0B9F0ACEC21
:100BD000AED00E94F22F01074C4F5354204348419E
:100BE0004E47455320592F4E203F000081D026F715
:100BF0000E94DC7943D270DE7093C801DDCF413FA3
:100C000049F46A2E7B2EADD0A62DB72D5092C80187
:100C10006FCED2CF4D3E09F5BF93AF937CD0A9F0F4
:100C2000ACEC85D00E94F22F010751554954205752
:100C30002F4F205341564520592F4E203F0058D06A
:100C400046F7A0911601A030E1F70E940A2DA0E01E
:100C50000E941D2DAF91BF910895443FE1F45BD0F8
:100C600029F40E940A2D0E94FD2D0895A9E65FD067
:100C70000E94F22F010753415645204348414E47F9
:100C80004553204245464F52452052554E210000C3
:100C90000E94593291CF5091140152FD1CC053FD56
:100CA0001AC04C31C0F04038B0F4AF3171F05A2F57
:100CB000AFE10E94D8326A916983AA95A517D9F746
:100CC0004883A3955092C80113CE0E94D83248831E
:100CD0005092C8010DCE0CCE0E94D8325A2F5F31EF
:100CE00021F0498149935395FACF50E258830895F2
:100CF0000E945932493559F0493749F04A3E39F096
:100D00004E3439F04E3629F04D3E19F0F1CF68944B
:100D10000895E8940895A091C801A0320895A8E824
:100D200006D00E94F22F01054F4B00000895EF936B
:100D3000FF939927A09340010E94F22F01052020E4
:100D400020202020202020202020202020202020A3
:100D5000202020202020202020202000FF91EF9123
:100D60000895A0E00E94AB324A3E09F40895423E45
:100D700021F4A030B9F3AA95F5CF433E21F4AB306E
:100D800089F3A395EFCF403268F3403858F7488392
:100D9000AB3009F0A395E6CFC9ECD1E056E149911B
:100DA0000E94642E5A95D9F70E94372E4EE511D035
:100DB00016F04A95E1F7542F53954427451719F03B
:100DC00024D04395FBCF43E20E94642E0E94372E2D
:100DD0000895CF93DF935F936F93E894C4E3D2E0D9
:100DE00053E2459FC00DD11D50E26991613238F444
:100DF0005A95D9F76F915F91DF91CF9108956894DB
:100E00006F915F91DF91CF910895DF93CF934F93CF
:100E10005F936F93C1E3D2E053E2459FC00DD11DB4
:100E2000DF93CF93A39653E26A91613210F45A95FF
:100E3000D9F7CF91DF9149910E94642E5A95D9F745
:100E40000E94372E6F915F914F91CF91DF9108955E
:100E5000AF93BF93EF93FF934F93AEE0B2E0E8E719
:100E6000FEE04591403011F04D93FBCF4F91FF9143
:100E7000EF91BF91AF9108952045786974202020AB
:100E80004E616D6520202053617665202052656C8F
:100E90006F616420202052756E202000AF93BF93B5
:100EA000EF93FF934F93AEE0B2E0E4ECFEE04591A8
:100EB000403011F04D93FBCF4F91FF91EF91BF91D7
:100EC000AF91089520202020202020205072696EAC
:100ED00074202053656E64202020526563762020A4
:100EE00020204E6577202000AF93BF93EF93FF93B0
:100EF0004F93AEE0B2E0E0E1FFE04591403011F009
:100F00004D93FBCF4F91FF91EF91BF91AF9108951A
:100F10002041626F72742020202020202020202079
:100F200020202020202020202020202020202020C1
:100F300020202000D9DFACECFADE0E94F22F010560
:100F4000524543454956494E472E2E2E00002092C9
:100F50002E010E942C089927ECECE0934001E3ED70
:100F6000F1E0EE2EFF2E41E10E94ED335CE00E94A5
:100F700009344B31B9F14A33D1F70E9409344B316E
:100F800089F1403218F041935A95B9F7403228F070
:100F90000E9409344B3131F1F9CFEEE0F2E0EE2E50
:100FA000FF2E53E2EE2DFF2DB396EE2EFF2E0E9464
:100FB00009344B31B9F04032D0F3433299F006C0D6
:100FC0000E9409344B3171F0403248F041935A95F8
:100FD000B9F70E9409344B3129F04032D0F793958C
:100FE0009036F9F60895A3E2BA9FA1E3B2E0A00D0E
:100FF000B11D0895BF93AF93F6DFC8E7D1E053E288
:1010000049914D935A95E1F7AF91BF910895BF93E0
:10101000AF93E9DFC8E7D1E053E24D9149935A9588
:10102000E1F7409178014093E901409179014093C3
:10103000EA01AF91BF910895BF93AF934F935F9330
:10104000D2DF139640E250E24D935A95E9F75F9153
:101050004F91AF91BF910895DF93CF93BF93AF931B
:101060004F9340E2A1E3B2E0CDEFDCE04D93219756
:10107000E9F74F91AF91BF91CF91DF91DF93CF937C
:10108000BF93AF934F9341E0A1E3B2E0C0E3D42F0D
:10109000DA5010F0C395FCCFD65CCD93DD93C0E25F
:1010A000CD9390964395403689F74F91AF91BF917C
:1010B000CF91DF910895425245414B004F56455222
:1010C000464C4F5700444956494445202F30005361
:1010D00051522046524F4D203C3000434F4E535406
:1010E000414E5420544F4F204249470057524F4ED3
:1010F000472045585052455353494F4E0053594E7F
:10110000544158204552524F5200554E4B4E4F5766
:101110004E204B4559574F52440057524F4E47208F
:10112000464F524D415400424144204C494E454E99
:10113000554D424552004E45585420572F4F20469A
:101140004F520052455455524E20572F4F20474F73
:1011500053554200544F4F204D414E5920474F5355
:10116000554200544F4F204D414E5920464F52009A
:10117000493243204552524F5200554E4B4E4F5725
:101180004E204552524F520044464C415348204550
:1011900052524F52004F5554204F46204152524117
:1011A0005900494E434F4D504C45544520504152F3
:1011B000004B4559574F5244204953204D495353F2
:1011C000494E470057524F4E472042434F505920F7
:1011D000004F5554204F462053435245454E00433F
:1011E000414E4E4F54204352454154452046494CB0
:1011F00045004D454D4F52592046554C4C004649EF
:101200004C45204E4F5420464F554E4400504147C8
:1012100045204E4F5420494E2046494C45005041F0
:10122000474553204E4F5420494E2052414E47458A
:10123000004E4F5420494E20475241504849435395
:10124000204D4F4445004E4F5420494E20544558A0
:1012500054204D4F4445004E4F205553522046498F
:101260004C4500535243204F5554204F4620534382
:101270005245454E0044455354204F5554204F4647
:101280002053435245454E0057524F4E472053502E
:101290005249544500494F2044495341424C45442A
:1012A000004E4F204558544D454D0000BE3508F0C6
:1012B0000895BF9328D0B395BE35E1F7BDDEBF9149
:1012C000DDCEBE3508F00895BF93AF93AB2FAA953E
:1012D000BDE508D0BA95BA17E1F7B395ADDEAF9189
:1012E000BF91CCCEBF93AF93DF93CF937CDE1396A9
:1012F000ED01B0E2A991AAA3BA95E1F7CF91DF91F0
:10130000AF91BF910895BF93AF93DF93CF936BDEFF
:101310001396ED01B0E2ABA1A993BA95E1F7CF9195
:10132000DF91AF91BF910895BF93AF93DF93CF93B8
:101330005ADEED0193964E914132E8F34038D8F7EA
:10134000AC1BBC0B9A2F925097FD9927CF91DF9140
:10135000AF91BF910895CAEEDCE02A922A9280E014
:101360002F92AA27BB27442771917032E9F37C3171
:1013700021F4A191BB27719156C07E3121F4A19136
:10138000BB27719150C07D3121F4B191A191719130
:101390004AC07F3121F4B191A191719144C07C3157
:1013A00030F4572F4C2E5D2ECE2FDF2F63C07432BA
:1013B000C1F47191703320F07A3310F4705305C08A
:1013C000713468F0773458F47753B03148F4A2950B
:1013D000B2955A2F5F70A07FB52BA70FEACF23C01D
:1013E00029C0703350F17A3340F5403810F086E070
:1013F0002AC1AA0FBB1FF0F04A2E5B2EAA0FBB1FFB
:10140000C8F0AA0FBB1FB0F0A40DB51D98F0705323
:10141000A70FB21D78F0B7FD0DC07191703318F0B1
:101420007A3308F4E6CF4F3709F473D1AA93BA930D
:1014300040E89DCF85E007C144C07134E8F37B35B7
:10144000D8F76081613458F16B3548F54C2E5D2E2C
:10145000CE2FDF2F21970C2F1D2FE0ECFBE152E068
:101460007591703011F488E0EEC0703261F46991CA
:10147000683299F45F93452FAA27BB27EC2FFD2FE5
:10148000C42DD52D71CF6991671751F375917032C5
:10149000E9F75395C02FD12FE3CF87E0D4C0403870
:1014A00010F086E0D0C07154770FEF93FF93E0E91E
:1014B000FCE0E70FF21DA191B191FF91EF917191C5
:1014C000B2CF7D3251F44F3711F444274DCF20F481
:1014D000403210F04FE748CF6FC0783231F471E0FE
:1014E0007F93AA27BB27472F3FCF793209F05EC0F1
:1014F0005F91513019F0523011F403D153C0533081
:1015000011F413D14FC0543029F4CCD1803009F0FC
:101510009AC046C0553029F4B991A991B095A095CB
:101520003FC0563009F4DDC1573009F48DC2583040
:1015300009F49EC2593009F4B3C25A3009F4C9C241
:101540005B3009F4D1C25C3009F4D2C25D3009F4D9
:10155000D4C25E3009F4AEC2503109F40AC251312E
:1015600009F425C1523109F428C1533109F40EC2DE
:10157000543109F423C25F3009F410C3553109F422
:10158000BCC1563109F4D0C1573109F4D5C150302E
:1015900029F06ED0803009F056C0AACF86E00895B9
:1015A000AA93BA93AA27BB2742E0DECE4F3720F496
:1015B0004F3010F086E047C07C3361F471E2608107
:1015C0006E3319F472E2619142C06D3311F473E22B
:1015D00061913DC07E3339F474E260816D3311F462
:1015E00075E2619134C07D3311F476E230C07B3214
:1015F00011F470E32CC07D3211F471E328C0733212
:1016000011F472E324C07A3211F470E420C07F3206
:1016100011F471E41CC0753211F472E418C0763212
:1016200011F473E414C05F91503021F05F3130F059
:101630001FD0F9CFB991A9913197089586E05F91B4
:101640005030C1F3FCCF4F914030E9F708955F91DE
:10165000A72FB52FA07FB07FBA1720F009D0803018
:1016600091F7F5CF5F937F93AA27BB27472F7CCEB7
:101670005F934F9319910991B991A991513211F446
:10168000FED03AC0523221F4F3D0A150A17034C040
:10169000533221F4FCD0A150A1702EC0543211F469
:1016A000F6D02AC0553221F4EAD0A150A17024C04E
:1016B000563211F4DDD020C0503311F441D01CC09B
:1016C000513311F43CD018C0523319F4A02BB12B74
:1016D00013C0503411F43FD00FC0513411F4A7D0CF
:1016E0000BC0523421F4A3D0A22FB32F05C0533422
:1016F00019F4A023B12300C0AA93BA934F915F912C
:101700000895B991A99103D0AA93BA930895B7FF08
:101710000895A095B095A30DB21D089517FF0895E3
:1017200000951095030D121D0895B991A991AB2B49
:1017300029F0B7FBA1E0BB270EF41297E5CFF0DF4D
:101740002B2F2127A00FB11F27FD08952B2F212715
:1017500027FD82E008950CD0A22FB32FBF770EF49F
:10176000D8DF37FD03C0452B09F4089582E00895C2
:101770007AD0CDDFB19F402D512DA09F202D312D4E
:10178000A19F300D411D521DB09F300D411D521DB6
:10179000089508E611E0B03818F0A00FB11FFBCF94
:1017A000A017B10718F0A01BB10BFACF0895B9919B
:1017B000A9910AE5A01BB20902C0B991A991E9DF7C
:1017C000FF93EF93E2EEF9E70AE510E0A017B10707
:1017D00048F4E00FF11FEA1BFB0BA491EF91FF917E
:1017E000BB27DECE04EB10E0A017B10778F40AE5C2
:1017F00010E0E01BF10BEA0FFB1FA491EF91FF91AA
:10180000BB27A095B095A30DB21DCACE0EE011E086
:10181000A017B10728F4E00FF11FEA1BFB0BEDCF77
:101820000EE011E0E01BF10BEA0FFB1FD6CF212FDA
:10183000202B11F483E0089516D022273327442764
:1018400051E1441FAA1FBB1F5A9551F0221F331F9D
:101850004FEF201B310BA8F7200F311F40E0F1CFD5
:101860000EF457CF08952B2F212727FB50DF56CF9B
:101870000A271B27AA27BB27012B89F00895B058F8
:101880001058A01BB10BAA27BB2748F00895B058E9
:1018900010580A1B1B0BAA27BB2708F00895A1E0CC
:1018A000B0E00895B991A99184E0B7FD08950F9330
:1018B0001F932F933F9388270A2F1B2FB2E0AA274D
:1018C000232D3327021B130B20F0A3952B0F321D62
:1018D000F9CFBB27AA93BA933F912F911F910F91F4
:1018E00008954F935F930E9481341991099142DFCB
:1018F000A42FB52F5F914F9153CE199109910230CA
:1019000039F420925001A2E0A0933301BB2748CEC6
:10191000013031F4A0913301A03011F43092330141
:10192000A0913301BB273CCE199109910EBD0E94B5
:101930000818AEB5BB2734CE10913E01103011F01F
:101940008CE1089519910991A4ECB2E00A171B07E4
:1019500010F082E10895FF93EF93FDE0ECE3E00FD8
:10196000F11F68940E942034EF91FF91A42FBB27B0
:1019700017CEB991B0937301A991A0937201CF933F
:10198000DF930E940C18DF91CF910ACEB991A991F3
:10199000BF3F71F0A09358010E944420803021F095
:1019A000AFEFBFEF8827FCCDA42FBB270C94D00A44
:1019B0000E9449208827B42FAA27F2CDB991A99176
:1019C000BF3F21F5A0FD11C0DF93CF93FF93EF93AD
:1019D0000E944120803019F08827CC27DD27DE01C6
:1019E000EF91FF91CF91DF91DBCDDF93CF93FF9309
:1019F000EF930E944120803019F08827EE27FF27BF
:101A0000DF01EF91FF91CF91DF91CACDA0935801F3
:101A10000E944420803021F08827AA27BB27C0CD10
:101A2000DF93CF937F9377270E944C20DF3F41F4D1
:101A3000CF3F31F4A72FBB277F91CF91DF91B0CD5E
:101A40007395703889F7F6CFA991A991A770A06C0A
:101A5000A0937C00A0917A00A064A0937A00A0914A
:101A60007A00A6FDFCCFA0917800B091790098CDC6
:101A7000B991A991B03061F4AF3F79F0A770A39507
:101A8000B0B1B695AA95E9F7AA27AA1FBB2788CDBA
:101A9000BA2FA0B1AB23BB2783CDA0B1BB2780CD8C
:101AA000B991A99171E00E9421398030C9F4BB2716
:101AB000A52F76CDB991A991CF93DF93CA2FDB2FB4
:101AC0000E945E39DF91CF91803051F4BB27A42F63
:101AD00067CDA99179910E943C39803009F460CD9D
:101AE000AA27BB278FE0ABCDB991A991BB2758CDD1
:101AF000B991A991AB2FBB2753CD0F93B991099100
:101B0000AA27BB27003019F4A091160145C0013067
:101B100029F4A0911601A030E1F33EC0023039F45F
:101B2000A0911601A030E1F7A091170135C0033054
:101B300019F4A091140130C0043039F4009114015B
:101B400000FD119602FD119727C0053039F4009170
:101B5000140101FD119603FD11971EC0063049F4D2
:101B600000911601023E09F41197033EA9F4119663
:101B700013C0073049F400911601043E09F4119690
:101B8000053E51F4119708C01F93109116010117DB
:101B9000E1F71F91A02FBB270F9102CDB991A99119
:101BA000BB27A13021F4A0916D01A395F9CCA230FF
:101BB00021F4A0916E01A395F3CCA0916F01F0CC1C
:101BC0004142532053474E20535152204E4F5420F0
:101BD000524E442041444320494E20585045454BE5
:101BE0002054454D50204C4F204849204B4559200A
:101BF000455045454B204552522041522053494EB5
:101C000020434F53204654595045204653495A4586
:101C1000205053544154205350492000FCE0E0E947
:101C2000A0E0B4EBA193BA95E9F7F1E0E8E6B0E102
:101C3000A193BA95E9F7FDE0ECE3B0E0A193A1939D
:101C4000A193BA95D9F7DD24CC2420920F012092DC
:101C50000D01AEE0A0932C01ACE3A0934401AEE2F1
:101C6000A0934501AFEFA09377010E94FD2D209234
:101C70005001A2E0A0933301A6ECA0937A0040911A
:101C80003D0140933A01409337010E9415799C2D04
:101C90000E9431791FD0803039F4AC2DAF35B8F3C4
:101CA0009CE0209250010895C0926D01D0926E0187
:101CB00080936F0120925001409177014F3520F4BD
:101CC000DD24C42E8827E3CF9CE0209250010895A4
:101CD000F70129C0F1E0E0EA20922A018827AD2D22
:101CE000BB27AB1701F171917F3FC1F17C31C9F086
:101CF0007E31B9F07D31A1F07F3191F0773271F111
:101D0000723241F471917F3F49F1773239F1723289
:101D1000C9F7E9CF7A3339F7B395AB1721F703C089
:101D200071917191E0CF70912D0170FF05C081E03C
:101D30007E7F70932D01089572FF0BC0AB7F70936F
:101D40002D01A0913E01A53011F0A03011F40E94A8
:101D50006C1B0E94FD3271917F3F19F4DD24C39406
:101D6000089577FD2BC07032F1F27A3311F4D394D9
:101D7000DACF773299F37134D8F07B3528F070528E
:101D80007134B0F07B35A0F4672E0E9447177D3385
:101D900079F4E1DA803069F4762D7154770FDCE064
:101DA000C0E9C70FD21DA993B99393CFEF91FF91CB
:101DB00087E00895703810F487E08ACF7F01E5EE60
:101DC000FEE07F73E70FF21D099445C0EDC0A0C28D
:101DD00036C10CC1EDC22EC33BC736C337C33BC3AC
:101DE0003EC38BC6A9C64CC3A2C3D4C2FAC32AC47D
:101DF00078C16CC47CC481C4E9C195C286C491C455
:101E000098C459C54AC1D5C077C22BC1E1C49BC48F
:101E100026C3E2C403C54EC2DDC2C4C5A7C716C6E9
:101E200022C627C673C1A7C6F6C678C728C637C656
:101E30005AC214C557C61FC181C297C300C392C4FA
:101E400098C43DC175C13BC692C188E0089584E144
:101E5000089583E108950E944B179CE0732C209213
:101E60002A01B191B032E9F3BA3311F0BF3F59F40E
:101E7000319770FC0E94372E40912A01443010F0B7
:101E80000E94E13826CFBB3311F47724EACFBC326D
:101E900091F440912A01403031F40E94632EBA2D12
:101EA000B770D9F706C00E94632EB0912B01B770AE
:101EB000D1F77724D6CF732CB332C9F420925801CE
:101EC0002092590148DA4A2F40932A01443018F4ED
:101ED000433001F4C6CF0E94E538683051F5509187
:101EE0002A015E7F0E94E738683119F5BACFB03415
:101EF00011F59DD740912A01433018F40E940B3010
:101F0000B0CF39F4A0935801B0935901A0932B019D
:101F1000A8CF5FEF0E94E738683259F45A2F0E9429
:101F2000E738683231F45B2F0E94E738683209F4F1
:101F300098CF8FE00895B13229F40DDA9A2F91CF1E
:101F400097CF8FCFB23241F441914F3FC9F3423224
:101F5000C1F30E94642EF8CFB63291F4FCD9B330AD
:101F600010F082E10895CCE3DDE0CA0FDB1F499158
:101F7000403029F00E94642E1196B330C0F371CF27
:101F8000B53229F4E8D94A2F0E94642E6ACF3197DE
:101F9000E2D9803009F00895903818F40E948D2D10
:101FA00060CF0E94E82D5DCFA0E0F3D60E94FD2D0A
:101FB0008FCEA2E0EED6A030C1F0A13059F0A091B2
:101FC0005A01A770AA0FB0912C01B770A295BA2B35
:101FD000B0932C01A0915801A770AA0FB0912C01C9
:101FE000B07FBA2BB0932C0173CE33CFA3E0D1D600
:101FF000A33018F1A0915801B0915901A09372013A
:10200000B0937301A0915A01B0915B01A093580164
:10201000B0935901A0915C01B0915D01B03011F411
:10202000A03051F00D010E940C180E94A017D001A1
:10203000803021F41197F2CF4BCE0BCF0895A5E05D
:10204000A8D6A43068F0B3D77F93E0D6E0936B01B5
:10205000F0936C010E941F317F9170932C0138CE58
:10206000F8CEA1E096D6A130D8F340915801417046
:1020700040930D012DCEA5E08CD6A43068F097D703
:102080007F93C4D6E0936B01F0936C010E944131C1
:102090007F9170932C011CCEDCCEA5E07AD6A430C3
:1020A00068F085D77F93B2D6C0936B01D0936C0153
:1020B0000E941C367F9170932C010ACECACEA5E0F7
:1020C00068D6A43068F073D77F93A0D6C0936B0115
:1020D000D0936C010E946C367F9170932C01F8CDE7
:1020E000B8CEA3E056D6A23080F061D77F93B091EE
:1020F0005801A0915A01A0936B01B0936C010E940A
:102100001E307F9170932C01E3CDA3CEA5E041D684
:10211000A43068F04CD77F9379D6E0936B01F093AD
:102120006C010E94FB317F9170932C01D1CD91CE37
:10213000A0913E01A03011F08CE10895A1E029D6D4
:10214000A130A8F3A0915801B0915901CCE3DDE092
:10215000CA0FDB1F40912C014F93AF92BF920E9498
:10216000B336BF90AF904F9140932C01B1CDA09169
:102170003E01A03011F08CE1089572D6C093700139
:10218000D093710184D67C32F9F4A1E003D6A1305A
:1021900070F2A0915801B0915901CCE3DDE0CA0F73
:1021A000DB1F40912C014F93AF92BF920E94DC360F
:1021B000BF90AF90C0917001D09171014993299265
:1021C0004F9140932C0184CD87E082CDA0913E01B8
:1021D000A03011F08CE1089543D6C0937001D093E4
:1021E000710155D67C3281F7A1E0D4D5A13009F038
:1021F00030CEFF93EF93AF92BF9240912C014F935B
:102200007F934F7040932C010E94D119C1E0D2E01E
:10221000ECE1F5E10E949531C0912C01C295C0938B
:102220002C010E94F22F03020000A0915801B091EE
:102230005901CCE3DDE0CA0FDB1FA6E14991403232
:1022400030F0403820F40E94642EAA95B9F7772721
:1022500061E025D00E94F719623079F4C0917001D5
:10226000D0917101799329927F914F9140932C01E4
:10227000BF90AF90EF91FF912BCD7F914F91409305
:102280002C01BF90AF90EF91FF91C0917001D09160
:1022900071014FEF499349931BCD87E019CD0E94FF
:1022A000EB178827603009F408950E94071E8827DD
:1022B00062E00895A3E06DD5A230A0F078D67F93B8
:1022C000D0916C01C0916B01F0915801E0915A01DD
:1022D000E0936B01F0936C010E94FB317F9170934E
:1022E0002C01F6CCB6CDA4E054D5A43021F48ED583
:1022F0000E94F730EDCCADCDA1E04BD5A13090F0F0
:10230000A0915801A295AA0FAF7EA0930F01E0CC37
:10231000A1E03FD5A13030F0A0915801A150CA2EC4
:10232000DD24089596CDA1E034D5A130D8F3A09155
:102330005801A150A0937701CBCC8BCDA5E029D536
:10234000A23030F1F1E0E0915801E770B0915A010C
:10235000B770BB0FB295B193A230C9F0E770B091DE
:102360005C01B770BB0FB295B193A33081F0E770F9
:10237000B0915E01B770BB0FB295B193A43039F044
:10238000E770B0916001B770BB0FB295B193A0CC6C
:1023900060CD5FCDA1E0FDD4A130D8F3A09158016C
:1023A000A53009F0A3700E941D2D0E94FD2D90CC38
:1023B000A1E0EFD4A13068F0A0915801B09159018B
:1023C000B03019F4A03009F483CC0E943032119758
:1023D000F7CF3FCD20925001A2E0A0933301A3E0BC
:1023E000D8D4A33020F1CCE3DDE0A0915801B09126
:1023F0005901B330E8F4AC0FBD1FA0935201A09374
:102400005401B0935301B0935501A0915A01B0917A
:102410005B01B33068F4AC0FBD1FA0935601B093BD
:102420005701A0915C01A09350012092330150CC40
:1024300082E14ECC20925001BF91BF9108952DD5DD
:10244000AB2B09F48BCC45CC26D543CCF701EFD48C
:102450000E940B303ECC21D50E9439323ACC672FF6
:102460006F931BD56F914A2F0E94642E65FD0E94C9
:10247000E1320ED57C3271F70AD50E94AB09F3CF59
:10248000A2E087D4A13019F0A23021F1E2CCA091D2
:102490005801AA95AF3510F08AE01ACCB0916F01BF
:1024A000BF3010F08DE014CCAF93CCEEDCE0A5E0B3
:1024B000AB9FC00DD11DB395B0936F01BD2DB395EA
:1024C000B068B993BC2DB993B0913D01B993DD24A7
:1024D000CF900895A0915A01AA95AF35E8F6B09132
:1024E0005801BA95B770B0933701B0916F01BF3002
:1024F00010F08DE0EDCBAF93CCEEDCE0A5E0AB9F30
:10250000C00DD11DB395B0936F01BD2DB395B068CB
:10251000B993BC2DB993B0913A01B993DD24CF9012
:102520004091370140933A010E9415790895B3D440
:10253000B0916F01B03011F48CE00895BA95CCEEF3
:10254000DCE0A5E0AB9FC00DD11DB0936F01B99148
:10255000B7FFF2CFBF77DB2EC990499140933A0184
:102560000E941579089587E0089595D490D4713428
:10257000D0F37B35C0F77154770F672E88D47D3345
:1025800091F70E94AB09803009F00895DCE0C0E9C2
:10259000C60DD21DA993B9937AD4743521F77191E0
:1025A0007F3409F70E94AB094A2E5B2E803009F078
:1025B0000895B0916F01BF3010F08EE00895CCEE19
:1025C000DCE0A5E0AB9FC00DD11DB395B0936F01CA
:1025D000BD2DB395B993BC2DB99369924992599287
:1025E00078CB59D4B0916F01B03011F48BE00895DD
:1025F000BA95CCEEDCE0A5E0AB9FC00DD11DB99142
:10260000B7FDF4CFBF77B0936A0159907991BCE0E0
:10261000A0E9A70FB21D0D911D91030D121D1E9370
:102620000E93A991B99111960A1741F41B1731F431
:10263000B0916F01BA95B0936F014BCBC52CD09080
:102640006A010895A0913E01A03011F08CE1089537
:1026500022D4BFEFB0937801B191B032E9F34B2FA0
:10266000BF3F21F40E94372E319733CBBA33D1F3D9
:10267000BB3391F3BC3231F40E94632EBA2DB77094
:10268000D9F7EACFB23241F441914F3F59F3423288
:1026900019F30E94642EF8CFB134B0F0BB35A0F42A
:1026A000B154BB0FB0936A01B081B13418F0BB359F
:1026B00008F40AC0F5D3DCE0C0E910916A01C10F4B
:1026C000D21DA993B993C8CF87E00895E6D380308F
:1026D00009F0FFCA4A2F4B2BE1F340912201403011
:1026E000E1F3409122014030E1F71197F3CFD5D3C8
:1026F000A0932301B0932401EDCFB2D3A091230185
:10270000A993A0912401A993E4CAC7D34A2F0E9498
:10271000ED33BED37C3221F4BAD30E94AB09F6CF9D
:10272000D8CA0E94F933A42FBB279AD3A993B9938F
:10273000D0CAF70188D34A2FD73020F4C03D10F417
:102740000E946739C6CAF7017ED35A2FAC2FBD2F1E
:1027500071E00E942F390E9430320E9430320E9474
:102760003032B7CA70910C0174FD30C096D3A1B954
:10277000B0CA70910C0174FD29C0F70164D3D03048
:10278000B1F4BC2FB770B39577276FE7A0FD70E861
:10279000A0FD6FEF77FB770F70F967FB660F60F9AD
:1027A000BA95C1F702B1072B062302B992CAD130FC
:1027B00041F4B2B1C095BC23C095CA23BC2BB2B9B9
:1027C00088CAD230E9F70E94F91783CA82E20895D5
:1027D00064D30E94E5337DCA43D3C0937001D09384
:1027E000710109911991105852D37C32A9F42BD35D
:1027F000B058D058C017D10710F00C2F1D2FA017BC
:10280000B10710F40A2F1B2FD0917101C0917001F4
:102810001058099319935DCA86E00895A0913E016E
:10282000A03011F08CE108951BD3C0937001D093B8
:1028300071012DD37C3281F7FAD2C8ECD1E07EE170
:102840007B9FC00DD11DCA0FD21DBB27A881D0917F
:102850007101C0917001A993B9933BCAA0913E0147
:10286000A03011F08CE10895FBD2C0937001D09399
:1028700071010DD37C3281F6DAD2C8ECD1E07EE171
:102880007B9FC00DD11DCA0FD21DA2EBCA0FA2E0C3
:10289000DA0FBB27A881A695BA2FA777B295B07893
:1028A000AB2BBB27D0917101C0917001A993B99353
:1028B00010CA86E00895D4D2C0937001D0937101FC
:1028C000E6D27C32B1F7B3D2C8ECD1E070913E01D0
:1028D0007370703021F5AF93BF93A695B6957EE1E6
:1028E0007B9FC00DD11DCA0FD21D7881BF91AF91C2
:1028F000A0FD7695B0FD7695B0FD7695A2EBB2E0A1
:10290000CA0FDB1FAC9170FDA295A695A770BB27DF
:10291000D0917101C0917001A993B993DAC9713056
:10292000D1F4AF93A695A695A69575E17B9FC00DB2
:10293000D11DCA0FD21D7881AF91A2FD7295A1FD64
:102940007695A1FD7695A0FD76957170D1E0C72FA3
:10295000A881A295DACF7130F1F7AF93A695A6952D
:102960007EE17B9FC00DD11DCA0FD21D7881AF9132
:10297000A1FD7295A0FD7695A0FD76957370D1E0CE
:10298000C72FA881A295C1CFAF93A6957AE27B9F6E
:10299000C00DD11DCA0FD21D7881AF91A0FD7295D7
:1029A000A72FB3CFA0913E01A03011F08CE1089584
:1029B000A3E0EFD1A33080F0A0915801B09159016C
:1029C000B33010F082E10895B23039F4A73F28F017
:1029D00082E1089581E208953CCACCE3DDE0CA0FAC
:1029E000DB1FC0934601D0934901AC81A03091F325
:1029F000AE3180F7BB81B03069F3B73158F7C09181
:102A00005801D09159012596BA9F000C111C000C59
:102A1000111CC00DC11DD330E8F6D0915A01C091F0
:102A20005C01C0934801D0934B01CF3F51F0DF3F91
:102A300041F0CA0FCA95CE3138F4DB0FDA95D731A1
:102A400018F40E944E3744C986E10895A0913E01D2
:102A5000A03011F08CE108951ED2A0912D01A46048
:102A6000A0932D0136C9A0912901A062A09329014C
:102A700030C9A0912901AF7DA09329012AC9A3E003
:102A800088D1A33009F0E5C90E944420443111F0F7
:102A90008EE108950E9458208030D9F719C9A3E02B
:102AA00078D1A33009F0D5C90E944420443111F0F7
:102AB0008EE108950E945B208030D9F709C9A2E019
:102AC00068D1A23009F0C5C9A4E1A0935C010E94BD
:102AD0005220803009F4FCC808950E9455208030AF
:102AE00059F4F6C8A1E055D1A13009F0B2C90E944D
:102AF0004420443191F38EE10895A2E04AD1A230FE
:102B000009F0A7C9A0915801B091590140915A010B
:102B1000CCE3DDE0403041F0D395413029F0D3954E
:102B2000423011F082E108950E94CF390E94BE3AEE
:102B3000803009F00895CCC8A2E02BD1A23009F072
:102B400088C9A0915801B091590140915A01CCE334
:102B5000DDE0403041F0D395413029F0D39542304B
:102B600011F082E108950E94883A0E94EB3980308A
:102B700011F308954EC0F7013ED1A09374010E9455
:102B8000E5386830B9F790FF28C0592F0E94E73820
:102B9000603481F7A030C9F0DDE0CCE340917401EE
:102BA0004B0F4A1BC40FD21DA13039F00E94EB38E5
:102BB000603579F55883AA95EFCF0E94F0386835D3
:102BC00041F558830E94E13884C80E94EB385030A8
:102BD000A1F350937401A52FDFCF592F0E94E7383E
:102BE0006831B9F43A2FDDE0CCE3409174014B0F2A
:102BF0004A1BC40FD21D5881503011F4303031F0CF
:102C00000E94E738683229F4AA9569F70E94E138F2
:102C100060C88FE0089541D1A0935801B093590145
:102C200037D17C3249F4319632D1723231F031975A
:102C30000E94AB0985D1F4CF4CC87191723231F04A
:102C40007F3F21F0BB27A72F7BD1F7CF7081E8CF43
:102C5000A0913E01A03011F48DE10895A7E099D034
:102C6000B0915801B0934C01B13039F0B23009F154
:102C7000B33009F43CC085E10895A730E1F7C8E519
:102C8000D1E0BA81B0934901BC81B0934601BE81C5
:102C9000B0934A01B885B0934701BA85B0934B0110
:102CA000BC85B09348010E94A634803009F0089595
:102CB0000FC8A63001F7C8E5D1E0BA81B093490149
:102CC000BC81B0934601BE81B0934A01B885B093F0
:102CD0004701BA85B0934801BB85B0934B010E9470
:102CE000A634803009F008950C94680EC4CFA43047
:102CF000E9F7C8E5D1E0BA81B0934601BB81B09352
:102D00004901BC81B0934B01BE81B09348010E9440
:102D1000A634803009F008950C94680EA0913E010D
:102D2000A03011F08CE10895F7018DD0C0935801C7
:102D3000D093590150917401A51708F45A2FA8E7B0
:102D4000B1E0503071F04D91A0937501B0937601D0
:102D5000A42FBB27F5D0A0917501B09176015A95AB
:102D6000F0CFAA27BB27ECD00C94690EA0913E01AE
:102D7000A03011F08CE10895A1E00BD0A13040F01B
:102D8000A09158014A2F43700E941C380C94680E81
:102D900060C8F701A03009F40895DF93CF93C8E528
:102DA000D1E040E05A2F503029F4A42F7F01CF9179
:102DB000DF910895DF93CF934F935F930E94AB0908
:102DC0005F914F91CF91DF91893121F488277F0165
:102DD000A42F0895A993B99343955A95503019F3A8
:102DE00071917032E9F37C3229F33197A42F7F017E
:102DF000CF91DF910895A3E0CCDFA33009F5909146
:102E00005801B0915A01A0915C010895D0915801E8
:102E1000C0915A01F0915C01E0915E01C0934601BE
:102E2000D0934901E0934701F0934A010895A2E04D
:102E3000B1DFA23029F4B0915801A0915A01089550
:102E4000AF91AF9106C8A2E0A5DFA230C9F7C0914B
:102E50005801D0915901A0915A01B0915B01089598
:102E6000F70115D0713478F07B3538F47154770F51
:102E7000DCE0C0E9C70FD21D0895713620F07B3722
:102E800010F47156F4CF8F918F9187E0089571916E
:102E90007032E9F30895F7010895F7010C94AB0936
:102EA000EF93FF930E94C532EC2FFD2F00E00E94AC
:102EB000653270912D01713011F4872F08C04A3EA0
:102EC000C9F400937401003031F4AA27BB27882786
:102ED000FF91EF910895C8E7D1E0A191A9930A95D8
:102EE000E1F7A0E2A993AFEFA993E8E7F1E00E9430
:102EF000AB09EDCF4C3E49F40030C9F2AA940E94D0
:102F0000C532A0E2A8830A95D2CF403248F24B37AF
:102F100038F6AA2DAD3120F60E94642E0395C7CF56
:102F200092E0BB27AC2DA3950E948D2D4AE30E9411
:102F3000642EBB27AD2D0E948D2D0E94632E089517
:102F4000DF93CF93BF93AF93A0915801B0915901F4
:102F5000B33098F4CCE3DDE0CA0FDB1FAF91BF9133
:102F6000A883C0915801D09159012196C09358016E
:102F7000D0935901CF91DF910895B45090F0AA0FEA
:102F8000BB1FB33070F4CCE3DDE0CA0FDB1FAF91A1
:102F9000BF91A993B993C0915801D091590122963C
:102FA000E5CF82E1AF91BF91CF91DF91089570910C
:102FB0002C01A0FF0895A33059F450915C015F707B
:102FC000550F707F572B70912C0150932C01089551
:102FD00050916001F4CF0E945E20403011F46627CA
:102FE0000895409360010E944F20413009F0662708
:102FF0000895AF3F31F42C9A2CBCACE5ACBD3DBC80
:1030000008952CBCAF73A064ACBD3DBC2C98089552
:10301000BDB5B7FFFDCF0895509172014091730186
:10302000433038F4DDE0CCE3C50FD41FA991BB27B2
:1030300010C05050444058F0550F441F433038F4EE
:10304000DDE0CCE3C50FD41FA991B99102C082E1A4
:1030500008954091720150917301430D521D4093A8
:10306000720150937301803009F408954F914F918C
:103070000895A0EAB1E04FEF52E24D935A95E9F777
:10308000C8E9D1E040E25A91503211F44A95D9F79B
:10309000442EA0EAB1E0C8E7D1E04C0EA03C28F4F1
:1030A000C41518F44881403009F4089593D04F3F77
:1030B000E1F37AD04F3FC9F3403081F798D04030E8
:1030C00069F73DD0403051F70AD0403039F7499187
:1030D000413618F04B3708F440524D93DFCF48810A
:1030E000403320F04A3310F4405302C0442708957F
:1030F000642F772721964881403380F04A3370F45B
:103100004053660F771F0B01660F771F660F771FFF
:10311000600D711D640F721D2196EDCF703029F086
:103120004DE14D937D936D9308956A3020F04CE10D
:103130004D936D930895605D6D934CE108954881C2
:10314000443211F044270895662777272196588145
:103150005033F8F05A3310F450530BC05134C8F0C8
:10316000573410F4575305C0513698F0573688F449
:1031700057555F705295550F661F771F550F661F85
:10318000771F550F661F771F550F661F771F2196F4
:10319000DECF703029F04FE14D937D936D9308950C
:1031A0004EE14D936D9308954881423211F04427CA
:1031B000089521964D934991423219F44D9341E07F
:1031C0000895403029F442E24D934FEF4D93089516
:1031D0004D93F1CF4881473211F04427089521964D
:1031E0004D9349914030E1F74FEF4D930895FF9390
:1031F000EF93BF93AF935F93E4ECF6E40E01459138
:10320000403089F0689457E0A591AE3239F0B99119
:10321000B13608F0B052AB1709F0E8945A95A1F70F
:1032200016F0E001EBCF5F91AF91BF91EF91FF916D
:10323000403041F04D934F934881403211F4219634
:10324000FBCF4F910895CBE7D1E0A0EAB1E040E297
:10325000E0E24993EA95E9F7A097A03C29F04D9167
:10326000423010F04F3F11F429920895403220F07F
:10327000403810F486D0F1CF4C3121F4ED91FF2786
:1032800019D0EBCF4D3121F4FD91ED9113D0E5CF65
:103290004E3131F444E275D0ED91FF273CD0DDCFC3
:1032A0004F3131F444E26DD0FD91ED9134D0D5CF62
:1032B00050D0D3CFE8944FE24395E051F742E0F786
:1032C000E05FF84D403311F063D068944FE24395CE
:1032D000E85EF340E0F7E851FC4F16F0403311F0A0
:1032E00057D068944FE24395E456F040E0F7EC592C
:1032F000FF4F16F0403311F04BD068944FE24395E6
:10330000EA50E8F7E65F16F0403309F041D040E3B9
:103310004E0F3ED00895E8944F2F42954F7011F014
:1033200012D068944F2F4F700EF011F00CD06894AB
:103330004E2F42954F700EF011F005D068944E2F2D
:103340004F7001D00895405D4A3308F0495F20D0A6
:103350000895E4ECF6E45591503009F408954517CA
:1033600011F03796F8CF5F9357E045914E3209F050
:103370000FD05A95D1F75F915C3110F040E208D040
:1033800008954993CB3918F029924F914F910895A0
:103390004993CB3928F029924F914F914F914F91FA
:1033A0000895FF93EF93A0913E01A0936E01AA2789
:1033B0000E941D2DA0912C01A0936A01A0910F01E4
:1033C000A0936D01A0912A01A093690120922A0186
:1033D000E8ECF1E0CCE2D7E0BEE2AEE14191499306
:1033E000AA95E1F7BA95C9F7EF91FF910895FF9378
:1033F000EF93A0916E010E941D2DA0916D01A093ED
:103400000F01A0916A01A0932C01A0916901A093E2
:103410002A01ECE2F7E0C8ECD1E0DECFA0910C018C
:10342000A4FD35C0C6E0D4E0A9E4BFE441B158E052
:1034300040FDB99340FFA99346955A95C9F7C4E258
:10344000D4E0A0E3B1E340B158E040FDB99340FFC0
:10345000A99346955A95C9F7C8EBD6E0AFEABFE203
:1034600041B158E040FDB99340FFA99346955A9564
:10347000C9F7C6EDD6E0A0E8BEE440B158E040FD93
:10348000B99340FFA99346955A95C9F708950E94AC
:10349000F22F130020494F2044495341424C4544E8
:1034A00020000895452FA6E10E946E2D4F5B0E94DB
:1034B000642E4DE30E94642EA7E10E946E2DC0E9A8
:1034C000DCE0C50FD21DC50FD21DA991B9919DE0B9
:1034D0000E948D2D0895A3E10E940B30A5E0C62F18
:1034E000CA95AC9FCCEEDCE0C00DD11DA881A7FF32
:1034F0000AC00E94F22FFF43414C4C202000A981BA
:10350000AF770EC008950E94F22FFF464F52200061
:103510004A8146954F5B0E94642E0E94632EA981CA
:10352000BB27A39592E00E948D2D4AE30E94642E52
:10353000BB27A8810E948D2D089520920F01A7E03E
:103540000E946E2D0E94FD2D0E94F22F1200424912
:103550005420303132333435363700000E94F22F98
:103560001300444952000E94F22F14004C455600AB
:10357000A7E20E946E2D0E94F22F16002045786966
:1035800074200000A0E60E946E2D0E94F22F160605
:103590002020476F20200000A0E40E946E2D0E9492
:1035A000F22F160C2053746570200000A7E10E94D2
:1035B0006E2D0E94F22F16122056696577200000AA
:1035C000AEE6A0932B07A7E30E946E2D0E94F22F78
:1035D0001618202020202000A5E00E946E2D0E94B9
:1035E000F22F00004156522D4368697042617369A1
:1035F0006332204D4F4E2020202050004091370153
:103600004F5C0E94642E0E94F22FFF3A000092E06D
:10361000BB27AC2DA3950E948D2D0E94F22FFF3A5F
:103620000000BB27AD2DA3950E948D2DEBE7F1E0A7
:10363000C6EED1E0AEE141EFB191B03031F0BE8FD6
:103640004CAF4993AA95C1F706C0B0E2BE8F4CAF0C
:103650004993AA95D1F7A7E10E946E2DC0E0D4E06E
:10366000E1E1F0E10E94F7309DE050E0452F4C5F32
:10367000B42FAA270E940B3015DF53955D30B1F7A8
:10368000452F4950B42FA9E00E940B300BDF539512
:103690005A31B1F7A7E30E946E2DC3E1D4E0EDE10A
:1036A000F0E10E94F7300E94F22F0413535441437B
:1036B0004B3A00009927BB27A0916F010E948D2DE6
:1036C0006CE0C0916F01C61720F0C61BB4E0B60FC6
:1036D00002DF6A95B1F708954F935F936F937F93DD
:1036E000EF93FF93CF93DF93AF93BF93AF92BF92CC
:1036F0008F939F9356DEA7DD20DF2ED08827A091E1
:103700002D014D3E11F4A16011C0413F11F4AA27D3
:103710000DC0423F11F4A46009C0433F71F767DE5A
:103720000E945932AA270E941D2DE6CFA0932D0199
:10373000409116014030E1F75ADE9F918F91BF9082
:10374000AF90BF91AF91DF91CF91FF91EF917F91BA
:103750006F915F914F910895209217015FDE409124
:1037600017014030D9F30C94FD3220922A012092A7
:103770003E01A5E00E946E2DC0E0D0E0EDE1F6E153
:103780000E949531A0E50E946E2D0E94F22F010249
:1037900044464C4153482073697A653A20000E94A0
:1037A0005E204F3749F40E94F22FFF353132204B13
:1037B00069427974650011C04F3F41F40E94F22FB5
:1037C000FF31204D69427974650007C00E94F22FD5
:1037D000FF3020427974650013C00E944F204130B1
:1037E000D1F0E6E0FAE3E8940E942034413009F495
:1037F00034C0443009F4B9CF423099F733D0B5CF53
:10380000E2E4FAE3E8940E942034413009F425C050
:103810004430B1F7AACFEAECF9E3E8940E942034EF
:10382000413009F41AC0473019F40E943F1D9DCF62
:103830004A3011F417D099CF423011F46DD095CFA2
:10384000433019F40E94961D90CF443019F40E9421
:10385000E81D8BCF4530F9F688CFA0911601A03036
:10386000E1F708950E94CF364F466F726D61742064
:103870004D656469756D3F00413009F00895A6E219
:103880000E946E2DC2E0D8E0EBE1FCE00E945D31C9
:103890000E94F22F0903466F726D617474696E673E
:1038A0002E2E2E202020202020000E94F22F0B03FD
:1038B00000000E946120803001F50E94F22F090370
:1038C000466F726D617474696E672E2E2E20446F80
:1038D0006E652100A2E70E946E2D0E94F22F0B035D
:1038E000202020507265737320616E79206B65799A
:1038F000212020000E94593208950E94F22F0903CE
:10390000466F726D617474696E672E2E2E2045723B
:10391000726F72210000DECFA0E60E946E2DC4E01F
:10392000D8E0E9E1FDE00E945D310E94F22F090537
:10393000417661696C61626C653A00000E94F22F09
:103940000A0546696C65733A20009CE00E9441209C
:10395000DF93CF93DF010E948D2D0E94F22FFF2075
:103960002F000E945E20A42FB0E011960E948D2DA2
:103970000E94F22F0B05426C6F636B733A00AF919C
:10398000BF910E948D2D0E94F22FFF202F000E94D8
:103990004920A0EFA49FD0011197B03009F41397EC
:1039A0000E948D2DA6E00E946E2D0E94F22F0C0524
:1039B000202020507265737320616E79206B6579C9
:1039C000212020000E9459320895204578697420F2
:1039D00020496E666F204261636B75705265737427
:1039E0006F7252657363616E202020202020446531
:1039F0006C6574652020202020202020202020209D
:103A0000466F726D6174204578697420466F726DDF
:103A1000617420202020202020202020202052659A
:103A20007363616E20202020202020202020202071
:103A30002020202020202020202020202020202086
:103A4000202020457869742020202020202020205C
:103A50002020202020202020202052657363616ECA
:103A60002020202020202020202020202020202056
:103A700020202020202020202020202020207727E8
:103A80000BD1A4E00E946E2DC1E0D2E0ECE1F5E1A3
:103A90000E949531A0E40E946E2D0E94F22F030235
:103AA00044656C6574652066696C6500B0D0709380
:103AB0005801EAD24C3FD1F34CD1413019F4A72F31
:103AC0009CD2F3D208957727E7D0A4E00E946E2D10
:103AD000C1E0D2E0ECE1F5E10E949531A0E40E9462
:103AE0006E2DA0E1A0935C010E94F22F03025361AE
:103AF000766520500000ACD28AD070935801C4D2B1
:103B0000403E20F4403161F0F4D0DECFBAD2D03064
:103B100021F4CC3010F427D1D7CF6FD2B4D108958F
:103B20000CD1413089F669D2BAD108957727B4D043
:103B3000A4E00E946E2DC1E0D2E0ECE1F5E10E942C
:103B40009531A0E40E946E2DA2E1A0935C010E9439
:103B5000F22F03024261636B7570000058D07093BE
:103B6000580192D2403920F4423161F0C2D0DFCF07
:103B700088D2D03021F4C03610F4F5D0D8CF3DD261
:103B800001D20895DAD0413091F637D207D20895A4
:103B9000772782D0A4E00E946E2DC1E0D2E0ECE154
:103BA000F5E10E949531A0E40E946E2D0E94F22F53
:103BB00003024C6F6164205000004AD228D07093F9
:103BC000580162D2403111F0A2D0E3CF88D10895DC
:103BD000772762D0A4E00E946E2DC1E0D2E0ECE134
:103BE000F6E10E949531A0E40E946E2D0E94F22F12
:103BF0000302526573746F72650009D070935801A7
:103C000043D2423111F08ED0E4CFE0D1089577272E
:103C1000B5D00BD10E9459324D3E21F42FD14F9196
:103C20004F9108954A3E09F40895403E19F40FD18A
:103C30007727EECF413E21F40AD170916001E8CFA1
:103C4000443E49F4703031F302D17150472F4F7028
:103C50004F30F1F2DECF453E59F4409160014717F5
:103C600009F4D8CFF4D07395472F4F7089F2D1CF94
:103C7000463E29F4703170F2EAD07051C9CF473E08
:103C800051F4409160014F3031F04051471718F026
:103C9000DED0705FBDCFBECF0E945E20403019F4F1
:103CA0004F914F911BC0409360010E9430320E949F
:103CB0003032F5D1413019F04F914F9101C0089544
:103CC0000E94A6364F44464C415348206E6F7420E4
:103CD000666F726D61747465640008950E94A63603
:103CE0004F44464C415348206572726F7221000068
:103CF00008950E94A6364F43616E206E6F74207344
:103D0000617665206F6E20746869730008950E9463
:103D1000A6364F4E6F2042415349432066696C6579
:103D2000000008950E94A6364F4E6F204241434B3B
:103D300055502066696C650008950E94CF36C04FCB
:103D400076657277726974652066696C653F0000FC
:103D500008950E94CF364F44656C6574652066698E
:103D60006C653F0008950E94A6364F4E6F20737019
:103D7000616365206C656674000008955F936F93BE
:103D80007F93A72FA07FA0936C01A0916C01AF70CF
:103D9000AB5FBA2FA4E00E940B30A6E00E946E2D0C
:103DA000A0916C01BB2795E00E948D2D0E94632E8F
:103DB000A5E00E946E2DA0916C01A093580164D1E2
:103DC000ADD04F3F61F1A0916C01A093580140E04C
:103DD00040935A0142E040935C01882769D18030CA
:103DE00091F4CCE3DFE00E94632E5CE05F934991A5
:103DF000403808F04EE2403208F440E20E94642E5F
:103E00005F915A9599F7A0916C01A395A0936C01CD
:103E1000AF7009F0BACF7F916F915F9108955DE027
:103E20000E94632E5A95E1F7EECF4F935F93C4E162
:103E3000D5E0472F4F705EE1459FC00DD11D52EF79
:103E400047E159934A95E9F75F914F9108954F9350
:103E50005F93C4E1D5E0472F4F705EE1459FC00DF1
:103E6000D11D5CE044E059934A95E9F75AE043E1FB
:103E700059934A95E9F75F914F910895A0911601E2
:103E8000A030E1F70895709358014CE040935A0137
:103E900040E140935C0106D1803009F01FCF709360
:103EA000580190913D01E0E0F0E99770929540EC67
:103EB000949FE00DF11D40E04F9300E0CCE3DFE084
:103EC000159119930A95E1F740935A0142E0409306
:103ED0005C01F1D04F9143954C3071F7089590916A
:103EE0003D019770E0E0F0E9929540EC949FE00D81
:103EF000F11D40E04F9340935A0142E040935C0132
:103F000070935801D5D0CCE3DFE00E946B793296F4
:103F10004F9143954C3071F778940895403139F4BE
:103F20000E94F22FFF4241533A0040E1089542318E
:103F300039F40E94F22FFF4255503A0042E10895B1
:103F4000443139F40E94F22FFF5553523A0044E1B4
:103F50000895463139F40E94F22FFF4156523A003B
:103F600044E10895483139F40E94F22FFF4C4F4745
:103F70003A0044E108950E94F22FFF2D2D2D2D00CF
:103F80004FEF08957093580140E640935A0142E183
:103F900040935C0187D0803009F0A0CE7093580127
:103FA0004427E0E0F0E94F93CCE3DFE000241590F4
:103FB00019920A94E1F740935A0142E040935C0160
:103FC0007AD04F914395403671F7089540E0E0E094
:103FD000F0E94F9340935A0142E040935C017093A3
:103FE000580166D0CCE3DFE00E946B7932964F91A6
:103FF0004395403671F7789408954F93FF93EF936C
:10400000DF93CF93BF93AF9340912C014093610115
:104010004CE440932C01C6E0DAE0E7E1FCE00E94CA
:104020005D310E94F22F0B0757726974696E672029
:10403000646174612E2E2E004091610140932C0129
:10404000AF91BF91CF91DF91EF91FF914F91089583
:10405000CAE2CAE240913D01942F4F5C499340E28D
:1040600049934BE54993409129014F934068409310
:1040700029010E949D794DE549934F914093290173
:1040800008950E94703B08950E943C3C0E94FF39B5
:1040900008950E94AC3908950E942C3A08950E9418
:1040A0004B3B08950E94D13B08950E94443C0895E3
:1040B0000E94C43C08950E94653C08950E94BA394C
:1040C00008950E94DD3A0895A1E00E94E533209210
:1040D0002A0120923E01A7E00E946E2DC0E0D0E0B0
:1040E000EDE1F6E10E949531A0E70E946E2D0E945D
:1040F000F22F01024156522D436869704261736983
:10410000633220636F6E6669677061676500A7E060
:104110000E946E2D0E94F22F1401436865636B7339
:10412000756D3A20000014D144D078D0AAD0DAD0EE
:10413000E2EBF3E4E8940E942034413009F403C137
:10414000423059F440910C0151E0452740930C0155
:104150000E9407790E94A321E7CF433059F4409190
:104160000C0152E0452740930C010E9407790E9400
:10417000A321DACF443059F440910C0154E0452793
:1041800040930C010E9407790E94A321CDCF4530B6
:1041900059F440910C0158E0452740930C010E94CE
:1041A00007790E94A321C0CF4A3011F40E94E92967
:1041B0008BCFA6E00E946E2D0E94F22F03014B656B
:1041C00079626F617264206C61796F75743A000076
:1041D000A7E040910C01417009F4A1E70E946E2D07
:1041E0000E94F22F03124445202851574552545A39
:1041F0002900A7E040910C01417009F0A1E70E945D
:104200006E2D0E94F22F041255532028515745520B
:1042100054592900A7E00E946E2D0895A6E00E943F
:104220006E2D0E94F22F060153657269616C207039
:104230006F72743A0000A7E040910C01427009F4DB
:10424000A1E70E946E2D0E94F22F0612203132301B
:104250003020427073202000A7E040910C01427092
:1042600009F0A1E70E946E2D0E94F22F0712203262
:1042700034303020427073202000A7E00E946E2D61
:104280000895A6E00E946E2D0E94F22F0901493286
:104290004320706F72743A00A7E040910C014470A3
:1042A00009F4A1E70E946E2D0E94F22F091220202E
:1042B000313030206B487A202000A7E040910C017B
:1042C000447009F0A1E70E946E2D0E94F22F0A129D
:1042D0002020343030206B487A202000A7E00E9454
:1042E0006E2D0895A6E00E946E2D0E94F22F0C0103
:1042F00053504920706F72743A00A7E040910C014E
:10430000487009F4A1E70E946E2D0E94F22F0C1252
:104310002020202035204D487A202000A7E0409121
:104320000C01487009F0A1E70E946E2D0E94F22F47
:104330000D122020313536206B487A202000A7E06E
:104340000E946E2D0895A0911601A030E1F7089506
:10435000AA27BB27CC27DD27EE27FF27159042E0B1
:10436000149EA00DB11DC21DD21D459147E0149EA3
:10437000A00DB11DC21DD21DFE3881F7EE27F0EF52
:10438000459141E7149EB01DC11DD21D459147E0E6
:10439000149EB01DC11DD21DF03091F7BF93AF9395
:1043A000DE019FE00E94E82DAF91BF910E94E82DB1
:1043B0000895204578697420204B65796220205348
:1043C000657220202049324320202053504920206C
:1043D00020202020202020202020202020202020DD
:1043E0002020202020202020436C6F6E6520AEE02E
:1043F000A0932C01C1E0D4E0ECE1F1E10E945D3139
:104400000E94F22F050500000E9411020E94F22F67
:10441000060328632920323030362D38204A6F6554
:10442000726720576F6C6672616D0000A2EAA093FC
:104430002C010E94F22F0803202020202020446518
:104440006469636174656420746F202020202020DB
:1044500000000E94F22F0903466C6F7269616E2C96
:10446000204572696B20616E64204469616E612E23
:104470000000AEE0A0932C010E94F22F0B025468C2
:10448000697320736F667477617265206973206C3D
:104490006963656E736564000E94F22F0C04756E8B
:1044A00064657220746865207465726D73206F6630
:1044B0002074686520000E94F22F0D04474E55209D
:1044C0005055424C4943204C4943454E5345205694
:1044D0002E3220000E94F22F0E035573652069745E
:1044E00020617420796F7572206F776E2072697306
:1044F0006B210000A2ECA0932C010E94F22F100768
:1045000020505245535320414E59204B45592000CD
:104510000E945932089561E00E94093450911601B9
:104520005D3E09F408954531B1F790913D01E0E019
:10453000F0E99770929540EC949FE00DF11DCCE36B
:10454000DDE050E0459149935A95E1F7CCE3DDE099
:104550000E94C4380E940934509116015D3E11F347
:104560004630A1F76395CCEBDDE00E94C4380E9491
:104570000934509116015D3EA9F24630A1F76395CA
:104580006931E9F644E00E94ED33089590913D01D0
:104590009770E0E0F0E9929540EC949FE00DF11DFA
:1045A00045E10E94ED3360E06F93CCE3DFE00E94D1
:1045B000A138803041F0813051F1883241F145E13C
:1045C0000E94ED33F2CF46E00E94ED33CCEBDFE00A
:1045D0000E94A138803041F08130C9F08832B9F0B2
:1045E00045E10E94ED33F2CF0E946B7978943296C8
:1045F00046E00E94ED336F9163956C30A9F60E94FE
:10460000F9334430E1F746E00E94ED3308956F91AD
:10461000089561E00E940934509116015D3E09F44D
:1046200008954531B1F7A0E8762F7A95A79FE0016C
:10463000ACE3BDE070E80E945E394D937A95D9F7FE
:10464000CCE3DDE00E94C4380E9409345091160189
:104650005D3E31F34630A1F763956F3021F744E0BA
:104660000E94ED33089545E10E94ED3360E06F93C1
:10467000CCE3DDE00E94A138803031F0883201F1D6
:1046800045E10E94ED33F4CFA0E8762F7A95A79FFD
:10469000E001ACE3BDE070E84D910E9467397A9586
:1046A000D9F746E00E94ED336F9163956E30F9F6CD
:1046B0000E94F9334430E1F746E00E94ED3308955B
:1046C0006F91089502414253282E2E2E0353474ED8
:1046D000282E2E2E04535152282E2E2E054E4F5486
:1046E000282E2E2E06524E44282E2E2E07414443AD
:1046F000282E2E2E08494E282E2E2E2E0958504593
:10470000454B282E0A54454D50282E2E0B4C4F2831
:104710002E2E2E2E0C4849282E2E2E2E0D4B45596E
:10472000282E2E2E0E455045454B282E0F45525211
:10473000282E2E2E104152282E2E2E2E1153494E49
:10474000282E2E2E12434F53282E2E2E1346545908
:104750005045282E144653495A45282E1550535477
:104760004154282E16535049282E2E2E174D454EB3
:1047700055282E2E805052494E542E2E81434C5394
:104780002E2E2E2E82474F544F2E2E2E83424F58C0
:104790002E2E2E2E8441434F50592E2E8553594E86
:1047A000432E2E2E86454E442E2E2E2E8742434FCC
:1047B00050592E2E885448454E2E2E2E89504F5338
:1047C0002E2E2E2E8A4E4F54452E2E2E8B454D4981
:1047D000542E2E2E8C52524541442E2E8D5257521D
:1047E0004954452E8E474F5355422E2E8F524554D5
:1047F00055524E2E90564D4F44452E2E914E4558B3
:10480000542E2E2E92494E5055542E2E93504C4FCE
:10481000542E2E2E94574149542E2E2E95545345E6
:10482000542E2E2E96544745542E2E2E97465345E1
:104830004C454354984F4E4552522E2E9953505545
:10484000542E2E2E9A534745542E2E2E9B45504FB4
:104850004B452E2E9C4745545049582E9D43495256
:10486000434C452E9E434F4C4F522E2E9F424F524B
:104870004445522EA0464F4E542E2E2EA150554D3B
:10488000502E2E2EA258504F4B452E2EA359454D3B
:1048900049542E2EA44C494D49542E2EA54745541B
:1048A00043484152A644524157544F2EA7504C41C1
:1048B000592E2E2EA85350524954452EA9534352D7
:1048C0004F4C4C2EAA425245414B2E2EAB464153E3
:1048D000542E2E2EAC534C4F572E2E2EAD445241FB
:1048E000572E2E2EAE49434F4D4D2E2EAF444154E0
:1048F000412E2E2EB043544558542E2EB1465245CB
:1049000041442E2EB24657524954452EB343424F8E
:10491000582E2E2EB447455441545452B546444562
:104920004C455445B646424F582E2E2EB750414C5A
:1049300045545445B8464F522E2E2E2EB949462E78
:104940002E2E2E2EBA4449522E2E2E2EBB4F5554AB
:104950002E2E2E2EBC46434952434C45BD414C455C
:1049600052542E2EBE46435245415445BF41534BEF
:104970002E2E2E2EC03F2E2E2E2E2E2EC742432EF2
:104980002E2E2E2ECA4E4F2E2E2E2E2ECB454D2E97
:104990002E2E2E2ECC5252442E2E2E2ECD5257522B
:1049A0002E2E2E2ECE474F532E2E2E2ECF52455426
:1049B0002E2E2E2EC2474F2E2E2E2E2ED0564D2E60
:1049C0002E2E2E2ED2494E502E2E2E2ED3504C2E21
:1049D0002E2E2E2ED74653454C2E2E2EDC475058C9
:1049E0002E2E2E2EDD43492E2E2E2E2EDE434F4C04
:1049F0002E2E2E2EDF424F2E2E2E2E2EE44C494DE3
:104A00002E2E2E2EE54743482E2E2E2EE644544FB2
:104A10002E2E2E2EE85350522E2E2E2EED44522E98
:104A20002E2E2E2EEE49432E2E2E2E2EEF44412ECC
:104A30002E2E2E2EF14652442E2E2E2EF246575258
:104A40002E2E2E2EF44741542E2E2E2EF546444562
:104A50004C2E2E2EF750414C2E2E2E2EFC46434926
:104A60002E2E2E2EFE4643522E2E2E2E002E2E2E73
:104A70002E2E2E2EA0910801B0910901ED01E2EB3E
:104A8000F2E0CE0FDF1FF6EFE0910E01FE0F7F93F5
:104A90004F92EEE14E2E6991ED915491762F7295E1
:104AA000762757FD672768B9ED91000056FD76B966
:104AB000049055FD76B96991162E54FD76B912947D
:104AC000162653FD76B907FC61254A9452FD76B946
:104AD000502D712D41F760910F0168B94F907F9172
:104AE000EE91F0910E01F395FA3029F4FF27A0938F
:104AF0000801B0930901F0930E010C94202CA091B1
:104B00000801B0910901D0910001C0910101C29545
:104B1000DC0FDE7EE5E110900F01FD914D2FF0FDE1
:104B2000429548B900004D2FF1FD429548B900006B
:104B30004D2FF2FD429548B900004D2FF3FD4295EF
:104B4000000048B96D2F4D2FF4FD429548B9CD9125
:104B5000F5FD62955D2F68B9F6FD52956D2F4D2FCD
:104B600058B9F7FD6295C0FD4295000068B9FC2F69
:104B7000EA95B9F618B8EE91F0910E01F395F2307E
:104B800029F4FF27A0930801B0930901F0930E01C7
:104B90000C94202CA0910801B0910901D1E0FEE114
:104BA00010900F01ED91CE2FC370588158B9CE2FC0
:104BB000C695C695C3705881E29558B9CE2FC3707B
:104BC0005881CE2FC69558B9C695C3705881ED91BE
:104BD000CE2F58B9C3705881FA9541F718B8EE91A5
:104BE000F0910E01F395F33029F4FF27A09308010B
:104BF000B0930901F0930E010C94202CA0910801B0
:104C0000B09109010F9310900F01EAE2D1E0CD912C
:104C1000C6950C2FC295C770F881F8B9C02F000057
:104C2000C770F881000000000000F8B9CD91C6956A
:104C30000C2FC295C770F881EA9579F718B81197CB
:104C40000F91F0910E01F395F43029F4FF27A09312
:104C50000801B0930901F0930E010C94202CA0914F
:104C60000801B0910901D0910001C0910101C295E4
:104C7000DC0FDE7EE0E110900F01FD914D2FF0FD85
:104C8000429548B90000000000004D2FF1FD42950B
:104C900048B90000000000004D2FF2FD429548B9D0
:104CA000000000004D2FF3FD4295000048B90000C0
:104CB00000006D2F4D2FF4FD429548B90000CD91B5
:104CC000F5FD62955D2F68B900000000F6FD529574
:104CD0006D2F4D2F58B9F7FD6295C0FD429500002C
:104CE000000068B9FC2F00000000EA9551F60000B2
:104CF00018B8EE91F0910E01F395F33029F4FF27E7
:104D0000A0930801B0930901F0930E010C94202C9C
:104D1000A0910801B0910901C0914101D82DF6EF91
:104D2000E0910E01FE0FE395E0930E01EA3088F169
:104D3000EC3069F59396A0930801B0930901209295
:104D40000E01DC3031F4D0914001D09341010C943C
:104D5000202CD83189F4A1E3B2E0C0912E01D3E236
:104D6000CD9FA00DB11DCFE0A0930801B093090124
:104D7000C09341010C94202CD83D49F4CBE4AEE023
:104D8000B2E0A0930801B0930901C09341010C94D3
:104D9000202C0F931F932F93D83D28F4DC2F0C2F3A
:104DA0001C2F2C2F05C029E61DE208E8DCECCBE423
:104DB0006C2F7C2F7295ED91E7FD6727EF7754916B
:104DC000ED9168B9172E56FD16B86C2F7C2F729591
:104DD00055FD16B8E7FD672754FD16B8EF770000BC
:104DE00053FD16B8049052FD16B8502DED9168B9D8
:104DF000172E56FD16B86C2F7C2F729555FD16B8E0
:104E0000E7FD672754FD16B8EF77000053FD16B88D
:104E1000049052FD16B8502DED9168B9172E56FD2D
:104E200016B86C2F7C2F729555FD16B8E7FD6727D5
:104E300054FD16B8EF77000053FD16B8049052FDEC
:104E400016B8502DED9168B9172E56FD16B86C2F77
:104E50007C2F729555FD16B8E7FD672754FD16B8EF
:104E6000EF77000053FD16B8049052FD16B8502D90
:104E7000ED9168B9172E56FD16B86C2F7C2F7295E0
:104E800055FD16B8E7FD672754FD16B8EF7700000B
:104E900053FD16B8049052FD16B8502DED9168B927
:104EA000172E56FD16B86C2F7C2F729555FD16B82F
:104EB000E7FD672754FD16B8EF77000053FD16B8DD
:104EC000049052FD16B8502DED9168B9172E56FD7D
:104ED00016B86D2F7D2F729555FD16B8E7FD672723
:104EE00054FD16B8EF77000053FD16B8049052FD3C
:104EF00016B8502DED9168B9172E56FD16B86D2FC6
:104F00007D2F729555FD16B8E7FD672754FD16B83D
:104F1000EF77000053FD16B8049052FD16B8502DDF
:104F2000ED9168B9172E56FD16B86D2F7D2F72952D
:104F300055FD16B8E7FD672754FD16B8EF7700005A
:104F400053FD16B8049052FD16B8502DED9168B976
:104F5000172E56FD16B86D2F7D2F729555FD16B87C
:104F6000E7FD672754FD16B8EF77000053FD16B82C
:104F7000049052FD16B8502DED9168B9172E56FDCC
:104F800016B86D2F7D2F729555FD16B8E7FD672772
:104F900054FD16B8EF77000053FD16B8049052FD8B
:104FA00016B8502DED9168B9172E56FD16B86D2F15
:104FB0007D2F729555FD16B8E7FD672754FD16B88D
:104FC000EF77000053FD16B8049052FD16B8502D2F
:104FD000ED9168B9172E56FD16B86D2F7D2F72957D
:104FE00055FD16B8E7FD672754FD16B8EF770000AA
:104FF00053FD16B8049052FD16B8502DED9168B9C6
:10500000172E56FD16B8602F702F729555FD16B8E5
:10501000E7FD672754FD16B8EF77000053FD16B87B
:10502000049052FD16B8502DED9168B9172E56FD1B
:1050300016B8602F702F729555FD16B8E7FD6727DB
:1050400054FD16B8EF77000053FD16B8049052FDDA
:1050500016B8502DED9168B9172E56FD16B8602F71
:10506000702F729555FD16B8E7FD672754FD16B8E9
:10507000EF77000053FD16B8049052FD16B8502D7E
:10508000ED9168B9172E56FD16B8602F702F7295E6
:1050900055FD16B8E7FD672754FD16B8EF770000F9
:1050A00053FD16B8049052FD16B8502DED9168B915
:1050B000172E56FD16B8602F702F729555FD16B835
:1050C000E7FD672754FD16B8EF77000053FD16B8CB
:1050D000049052FD16B8502DED9168B9172E56FD6B
:1050E00016B8602F702F729555FD16B8E7FD67272B
:1050F00054FD16B8EF77000053FD16B8049052FD2A
:1051000016B8502DED9168B9172E56FD16B8612FBF
:10511000712F729555FD16B8E7FD672754FD16B837
:10512000EF77000053FD16B8049052FD16B8502DCD
:10513000ED9168B9172E56FD16B8612F712F729533
:1051400055FD16B8E7FD672754FD16B8EF77000048
:1051500053FD16B8049052FD16B8502DED9168B964
:10516000172E56FD16B8612F712F729555FD16B882
:10517000E7FD672754FD16B8EF77000053FD16B81A
:10518000049052FD16B8502DED9168B9172E56FDBA
:1051900016B8612F712F729555FD16B8E7FD672778
:1051A00054FD16B8EF77000053FD16B8049052FD79
:1051B00016B8502DED9168B9172E56FD16B8612F0F
:1051C000712F729555FD16B8E7FD672754FD16B887
:1051D000EF77000053FD16B8049052FD16B8502D1D
:1051E000ED9168B9172E56FD16B8612F712F729583
:1051F00055FD16B8E7FD672754FD16B8EF77000098
:1052000053FD16B8049052FD16B8502DED9168B9B3
:10521000172E56FD16B8612F712F729555FD16B8D1
:10522000E7FD672754FD16B8EF77000053FD16B869
:10523000049052FD16B8502DED9168B9172E56FD09
:1052400016B8612F712F729555FD16B8E7FD6727C7
:1052500054FD16B8EF77000053FD16B8049052FDC8
:1052600016B8502DED9168B9172E56FD16B8622F5D
:10527000722F729555FD16B8E7FD672754FD16B8D5
:10528000EF77000053FD16B8049052FD16B8502D6C
:10529000ED9168B9172E56FD16B8622F722F7295D0
:1052A00055FD16B8E7FD672754FD16B8EF770000E7
:1052B00053FD16B8049052FD16B8502DED9168B903
:1052C000172E56FD16B8622F722F729555FD16B81F
:1052D000E7FD672754FD16B8EF77000053FD16B8B9
:1052E000049052FD16B8502DED9168B9172E56FD59
:1052F00016B8622F722F729555FD16B8E7FD672715
:1053000054FD16B8EF77000053FD16B8049052FD17
:1053100016B8502DED9168B9172E56FD16B8622FAC
:10532000722F729555FD16B8E7FD672754FD16B824
:10533000EF77000053FD16B8049052FD16B8502DBB
:10534000ED9168B9172E56FD16B8622F722F72951F
:1053500055FD16B8E7FD672754FD16B8EF77000036
:1053600053FD16B8049052FD16B8502DED9168B952
:10537000172E56FD16B8622F722F729555FD16B86E
:10538000E7FD672754FD16B8EF77000053FD16B808
:10539000049052FD16B8502DED9168B9172E56FDA8
:1053A00016B8622F722F729555FD16B8E7FD672764
:1053B00054FD16B8EF77000053FD16B8049052FD67
:1053C00016B8502DED9128B82F911F910F910C9484
:1053D000202C0E94CF366F436C6F6E6520737973FB
:1053E00074656D3F2000413009F0089565D087D085
:1053F000803079F078D00E94A6364F4E6F20636FD0
:105400006E74726F6C6C657220666F756E642000CE
:1054100008958DD0803069F066D00E94A6364F4E38
:105420006F204D65676136343420666F756E640099
:105430000895CBD09BD0EE27FF2750E060E0059089
:10544000B6D00590BBD063956038C9F79CD0539512
:10545000A9F74CEA4ED040EA4CD04AD046EE49D0AB
:105460000E9430320E9430320E9430324CEA41D0E9
:1054700048EA3FD03DD041ED3CD00E9430320E94FE
:1054800030320E9430324CEA34D044EA32D030D04C
:105490004CEF2FD00E9430320E9430320E943032C6
:1054A00022D00E94A6368053797374656D20636C98
:1054B0006F6E65640000089543E54CBD2DBC249AD1
:1054C0002C984FEF4A95F1F72C9A4FEF4A95F1F748
:1054D0002C984FEF4A95F1F72C984FEF4A95F1F73A
:1054E0000E94303208952C9A4CE54CBD3DBC089585
:1054F00044274EBD4DB547FFFDCF4EB508958827D3
:105500004CEAF7DF43E5F5DFF3DF433509F081E0EF
:10551000EFDF0895BF93AF934F93A42FBB270E9453
:10552000E82D0E94632E4F91AF91BF910895882777
:1055300040E3DFDFDDDF40E0DCDFDADF4E3111F0BA
:1055400082E0089540E3D5DFD3DF41E0D2DFD0DF52
:10555000463911F082E0089540E3CBDFC9DF42E035
:10556000C8DFC6DF493009F082E008954CEAC1DFA8
:1055700040E8BFDFBDDFBCDF0E9430320E94303226
:105580000E94303208954CE4B4DF452F4695B1DFD8
:10559000452F440F440F440F440F440F440F440F52
:1055A000A8DFA6DF0E9430320E943032089540E426
:1055B000A0DF9EDF462F9DDF402D9BCF48E499DF83
:1055C00097DF462F96DF402D94CF4F93FF93EF93B5
:1055D000DF93CF93BF93AF9340912C014093610130
:1055E0004CE440932C01C5E0DAE0E8E1FCE00E94E5
:1055F0005D310E94F22F0B06436C6F6E696E67205F
:1056000053797374656D2E2E2E0040916101409385
:105610002C01AF91BF91CF91DF91EF91FF914F910D
:10562000089528B818954F935F936F93FF93EF9366
:10563000DF93CF93BF93AF930F921F92FFB7FF9368
:1056400030921101B0913101B7FF5C98B7FD5C9ABF
:105650004B99BE7F4B9BB160B0933101C8E0D1E064
:105660005F89A889E9890A881B88A00DE11DA88B9C
:10567000E98BFFA14491AD89AF3F09F4452F5AA5AD
:105680004503B0E8B10DB093B300EE89FF89488DB2
:10569000598DAA27E2FDA095E5FDA095F4FDA09502
:1056A00057FDA095AA1FEE1FFF1F441F551FEE8B2D
:1056B000FF8B488F598F830C921CEBA9FF81EF233E
:1056C000E8B97894E9A190FC04C0F8A58F1608F415
:1056D00090C0FCE0E2FFFDEE8F1639F45E98E3FF28
:1056E000AFC0B2E8B0938000ABC0F1E1E2FFF3EFEE
:1056F0008F1639F45E9AE3FFA3C0B2ECB09380003A
:105700009FC0FBE1E2FFFFEF8F1621F4EFEFE09384
:105710003B0196C0F2E0E2FFF9EE8F1619F42092F9
:105720003B018EC0F9E3E2FFF7E08F1609F088C075
:10573000A8ECA883A1E0A9832E8288249924AAE05A
:10574000A9AFA5E0E2FFA39542E3E2FF4CE3BA8DE7
:10575000B395BA1731F4BB27EB8DFC8D3196EB8FE7
:10576000FC8FBA8FE885E395E41709F4EE27E88704
:10577000FDE8E0E0AC89EA0FF21DB491B21511F03A
:10578000A395AC8BBAA7A0915001A03009F458C0E2
:10579000B0915101B395B0935101BA17C0F3BB2733
:1057A000B0935101E0915201F0915301C091560123
:1057B000D09157012196A191E0935201F0935301AA
:1057C000AE3F09F056D6FD1798F0EC1788F0A0917F
:1057D0003301A13029F4A2E020925001A0933301BB
:1057E000E0915401F0915501E0935201F09353017F
:1057F00027C0A0918400AA3FE0F3AB3F00F0AC3F8C
:1058000000F0AD3F00F0AE3F00F0E5FD19C0E091C3
:105810002901E7FD0C948826E0913E01E53011F462
:105820000C942F26E37011F40C943A25E13011F416
:105830000C947F25E23011F40C94CA250C94FE25BB
:10584000A0911401A5FD23C0E091C000E7FF65C051
:10585000E091C600F5EFB491B0FF34C0A7FF03C0DC
:105860002092160157C0E33809F4E0E1F6E84091D0
:105870000C0140FDFE5FEF77A4FFA6FDF395A4FFAA
:10588000A0FDE068E491E0931501A06244C0E091BE
:105890001501E0931601E0931701EE3E19F4A2FD05
:1058A0000C94380040912D01E33611F4A2FD4160C3
:1058B000E03711F4A2FD4260EC3F09F444604093EC
:1058C0002D0128C0E03F11F4A06825C0E03E11F48E
:1058D000A06421C0E23121F4A160A7FDAE7F1AC00F
:1058E000E93521F4A260A7FDAD7F14C0E43151F485
:1058F000A6FD04C0A460A7FDAB7F0CC0A860A7FDF7
:10590000A77F08C0E13121F4A061A7FDAF7E02C0EE
:1059100020921601AF71A093140140910C0141FD3A
:105920000E94A17841FF0E94D678FF91FFBF1F908F
:105930000F90AF91BF91CF91DF91EF91FF916F9158
:105940005F914F911895AAEBA4B9AFEFA5B9A0EE5E
:10595000A7B9A0E0A8B9A0EFAAB9AFEFABB9A6B1BB
:10596000AF77A0932901B2ECB0938000B9E1B09376
:105970008100F4E0A2FFF4E0F0938700FEEFA2FFC5
:10598000F6EFF093860020928900FAE5F093880004
:10599000F4E0F0938B00F8EDF0938A00A6E0A0937A
:1059A0006F00A2E0A4BDA1E0A5BDA1E3A7BDA3E84F
:1059B000A093B000A1E0A093B100A0E8A093B30031
:1059C0002092B6002092C000A0E1A093C100A6E6FC
:1059D000A093C200ACE5B0910C01B3FDAFE5ACBD46
:1059E000A0E0ADBDA5E17AD0C8E0D1E0A8ECA993D4
:1059F000A1E0A993AEE12992AA95E9F7AAEAA093BA
:105A00001E01A093200120922A0120920D01AEE3F5
:105A1000A0931C010F93009129010F770093290196
:105A200006EE07C00F930091290100680093290139
:105A300004EE009330010F910895A0933E01A03031
:105A400041F4ACE3A0934401AEE2A0934501A6EE7D
:105A500042C0A13069F4A8EAA0934401A4E7A0934E
:105A60004501A0E0A0930001A0EEA093010124C095
:105A7000A23091F4A8E7A0934401ACE4A0934501BF
:105A8000C0E0D1E0A0E0A993A0E4A993A0EAA99383
:105A9000A0EEA993A3EE1FC0A33081F4A4E5A093C8
:105AA0004401AAE3A0934501C0E0D1E0AA27B8E0F1
:105AB000A993A05EBA95E1F7A7EE0DC0A0E8A09368
:105AC0004401A0E4A0934501A0E2A0930001A0EE50
:105AD000A0930101A0ECA09330010895AA0FAE7E1F
:105AE000A0932C010895A295AA0FA07EA0930F0168
:105AF000089548834091290147FD0EC0CF93DF935D
:105B00005F9342EBC40F42E0D41F40912C014E7EC4
:105B100048835F91DF91CF9108954F935F936F9387
:105B2000AF93BF9340E2592F5370523061F053301E
:105B300009F44BE2B7FF05C0A095B095A30DB21DC7
:105B40004DE20E94642E592F5C70692F6073E894B7
:105B50004FE24395A051B742E0F7A05FB84D5C30EB
:105B600009F42BD04FE24395A85EB340E0F7A8516B
:105B7000BC4F53FD22D0603309F4A3D04FE24395CC
:105B8000A456B209E0F7AC59BF4F503009F015D018
:105B9000603209F496D04FE24395AA50E8F70DD051
:105BA000A65F603109F48DD040E34A0F8DD0BF91DC
:105BB000AF916F915F914F910895403311F06894C8
:105BC00083C091FD81C0F6F390FF08957CC00895D5
:105BD0004F9390FF05C04B2F429509D04B2F07D014
:105BE0004A2F429504D04A2F02D04F9108954F700A
:105BF000405D4A3308F0495F67C040913E01403044
:105C0000B1F0AF93BF93CF93DF93D1E0C8ECACE595
:105C1000BEE12992BA95E9F7AA95D1F7DF91CF9124
:105C2000AA24BB2420922B01BF91AF910895AF937A
:105C3000BF93CF93DF93D1E0C8ECA7E1BEE14993D6
:105C4000BA95E9F7AA95D1F740912C014E7EA7E1CC
:105C5000BEE14993BA95E9F7AA95D1F7DF91CF91C3
:105C6000AA24BB2420922B01BF91AF910895AF933A
:105C7000BF9320922B01A0912A01A03051F4A7E1FB
:105C8000AA24B394AB1571F7B6E1BB2ECF93DF9383
:105C900062C0A13029F4BF91AF914AE00C94ED337A
:105CA000A23021F4BF91AF914AE090C4A33019F41F
:105CB000BF91AF910895BF91AF915AE00E94E7382C
:105CC00008954CE201C040E2AF93BF93A0912B0135
:105CD000A395A0932B01A0912A01A43030F0BF918D
:105CE000AF91542F0E94E7380895A030A9F0A33057
:105CF00059F4A42FBB275F936F930E94A0176F9155
:105D00005F91BF91AF910895BF91AF91A0912A018A
:105D1000A1FF0C94ED335AC4EF93E0913E01E030C3
:105D200009F09AC0EF91CF93DF932FD496FD35C041
:105D3000E0DEA395AE3131F4AA27B395B73111F463
:105D4000B6E107C0AA2EBB2EDF91CF91BF91AF91D4
:105D50000895AA2EBB2ED1E0C8EC4F93A6E1BEE178
:105D60004E8D4993BA95E1F7AA95C9F7AEE140E2A5
:105D70004993AA95E9F7D4E0CAE7A6E1BEE14E8DC2
:105D80004993BA95E1F7AA95C9F7AEE140912C0184
:105D90004993AA95E9F74F91D7CFAB31A8F6B23125
:105DA00098F6AD5FAA2EEF93FF934F925F926F929A
:105DB0007F9270F85F93E42FF6EFB5E0442455240A
:105DC00066245527A491A7FD539550FB40F8A6FDE6
:105DD000539550FB41F8A5FD539550FB50F8A4FD99
:105DE000539550FB51F8A3FD539550FB60F8A2FD6D
:105DF000539550FB61F8F3955527A491A7FD539552
:105E000050FB42F8A6FD539550FB43F8A5FD539572
:105E100050FB52F8A4FD539550FB53F8A3FD539546
:105E200050FB62F8A2FD539550FB63F8F395442DA7
:105E300060DE2196452D5DDE2196462D5ADE6C965C
:105E4000BA9509F0BBCF5F9170FA7F906F905F9029
:105E50004F90FF91EF9178CFFF93CF93DF936F93A4
:105E60007F93E42F60910D0160FD1EC0F6EFAA2D17
:105E7000BB2DDAE0C49137D0B395AA2D96FD33D06F
:105E800096FDB395F395AA2DDA95A1F7AA2DAA5FF1
:105E900096FDAA5FAA2E7F916F91DF91CF91FF911E
:105EA000EF91BF91AF910895FAE7EF77AE2FEEE350
:105EB000EA0FF21DAA0FEA0FF21DAA2DBB2DD6E0A4
:105EC000C49155D0B395AA2D96FD51D096FDB395AA
:105ED000D0FD3196AA2DDA9599F7AA2DAC5F96FDE3
:105EE000AC5FAA2ED8CF60912C016F936295C7FD4D
:105EF000629560932C01A2D0A39596FD9FD096FD4C
:105F0000A395C6FD629560932C0198D0A39596FD4C
:105F100095D096FDA395C5FD629560932C018ED01A
:105F2000A39596FD8BD096FDA395C4FD62956093D5
:105F30002C0184D0A39596FD81D096FDA395C3FD39
:105F4000629560932C017AD0A39596FD77D096FD4B
:105F5000A395C2FD629560932C0170D0A39596FD28
:105F60006DD096FDA3956F9160932C01089560917B
:105F70002C01D0FDC295762FC7FF729570932C012E
:105F80005DD0A39596FD5AD096FDA395762FC6FFBA
:105F9000729570932C0152D0A39596FD4FD096FD2B
:105FA000A395762FC5FF729570932C0147D0A395CA
:105FB00096FD44D096FDA395762FC4FF72957093FD
:105FC0002C013CD0A39596FD39D096FDA395609306
:105FD0002C0108954F934591403011F44F9108954D
:105FE00073DEF9CFFF91EF91EE0FFF1FAF93BF93D9
:105FF000B591BF3F11F0A5910ED0BF91AF914F93D6
:106000004591403031F44F913197F695E7953196AF
:1060100009945ADEF5CFEF93E0913E01E03021F094
:10602000EF91AA2EBB2E0895EF91AE3108F0ADE1AD
:10603000B73108F0B6E1AA2EBB2E0895CF93DF93B7
:10604000C0914401CA1728F0C0914501CB1708F050
:1060500003C0DF91CF910895AF93BF934F935F93A8
:10606000C0913E01C53021F0C37031F0C23008F458
:1060700041C009F464C081C051E0AC3360F5BE3268
:1060800050F5B0FD550FB0FD550FA0FD550FB6955D
:10609000A695CEE1BC9FD1E0C8ECCA0FD21DC00DC1
:1060A000D11DA2EBB2E0CA0FDB1FA881B0912C0179
:1060B000BE70B295A07EBA17A9F0B0912C01BE7047
:1060C000AB2BAE7EA883A2EBB2E0CA1BDB0BB88180
:1060D000B52BBF70B8835F914F91BF91AF91DF91A6
:1060E000CF910895A2EBB2E0CA1BDB0BB8815095AB
:1060F000B523EFCFCA2FC770C39540E00894441F63
:10610000CA95E9F7A695A695A695C5E1D0913E0159
:10611000D2FDC0E1BC9FD1E0C8ECCA0FD21DC00DBA
:10612000D11DA0912C01A695A17029F44095A881BC
:10613000A423A883D0CFA881A42BA883CCCFCA2F17
:1061400050912C015695537043E0C37031F0440FC9
:10615000440F550F550FCA95C9F74095A695A695BA
:10616000CEE1BC9FD1E0C8ECCA0FD21DC00DD11D3D
:10617000A881A423A52BA883AECFCA2F50912C01B0
:106180005E704EE0C17011F4429552954095A6950F
:10619000CAE2BC9FD1E0C8ECCA0FD21DC00DD11D10
:1061A000A881A423A52BA88396CFCE3108F0CDE1FA
:1061B000EE3108F0EDE1D73108F0D6E1F73108F023
:1061C000F6E1EC1718F40E2EEC2FC02DFD1718F485
:1061D0000F2EFD2FD02D0895EC1718F40E2EEC2F56
:1061E000C02DFD1718F40F2EFD2FD02D0895AF935D
:1061F000BF93CF93DF93EF93FF935F93D6DFAC2FE3
:10620000BD2FCF93DF93C3D1288252EBC50F52E04D
:10621000D51F50912C015883DF91CF91AE1711F00B
:10622000A395EFCFBF1719F0AC2FB395EACF5F91CD
:10623000FF91EF91DF91CF91BF91AF910895AF930F
:10624000BF93CF93DF93EF93FF935F93C5DFAC2FA3
:10625000BD2FF4DEA395AE17E1F7F0DEB395FB1783
:10626000E1F7ECDEAA95AC17E1F7E8DEBA95BD17C9
:10627000E1F75F91FF91EF91DF91CF91BF91AF91E6
:106280000895AF93BF93CF93DF93EF93FF935F9303
:10629000A3DFBD2FAC2FD2DEAE1711F0A395FBCF3D
:1062A000CDDEFB1711F0B395F5CF5F91FF91EF9124
:1062B000DF91CF91BF91AF91089599DFAF93BF93D5
:1062C000CF93DF93EF93FF934F935F936EDF4C2F4A
:1062D000BD2FAC2F5CD152EF599351EFA395AE1760
:1062E00011F05993FBCF53EF5993A42FB395BF17D8
:1062F00039F04DD150EF5993AE2F49D15993F5CF85
:10630000A42F45D154EF599351EFA395AE1711F037
:106310005993FBCF55EF59935F914F91FF91EF91B7
:10632000DF91CF91BF91AF910895C7DF5F93AF9396
:10633000BF93CF93DF93EF93FF9337DFBD2FAC2F46
:1063400026D15BEF59935CEEA395AE1711F05993EC
:10635000FBCF5CEF5993FF91EF91DF91CF91CF93FA
:10636000DF93EF93FF93BD2FAC2FB39510D15DEF6B
:10637000599350E2A395AE1711F05993FBCF5EEFFE
:106380005993FF91EF91DF91CF91CF93DF93EF93EB
:10639000FF93BD2FAC2FB395AF93F9D0A2EBB2E032
:1063A000CA0FDB1F50912C0152955E7E2196AF9152
:1063B000A395AE1711F05993FBCFFF91EF91DF91A9
:1063C000CF91CF93DF93EF93FF93BD2FAC2FBE5FA1
:1063D000DED05EEE59935DEEA395AE1711F05993A2
:1063E000FBCF5FEE5993FF91EF91DF91CF91BF917A
:1063F000AF915F9108950F931F932F933F93AF93A6
:10640000BF93CF93DF93DE010FEFCE1B10F4019506
:10641000C1951FEFDF1B10F41195D195CD1760F0DA
:1064200000C02C2F26950ADEAE1789F0A00F2D1B79
:10643000D0F7B10F2C0FF7CF2D2F2695FFDDBF170B
:1064400031F0B10F2C1BD0F7A00F2D0FF7CFDF913C
:10645000CF91BF91AF913F912F911F910F910895CF
:10646000AF93A82DA73EE9F3A82DA73EE9F7AF917A
:106470000895EF93FF93AF93A0931D01FBE8A6FD52
:10648000FCE8F0932F01AF73AA0FFDE8E0E8EA0FF4
:10649000F21DA591A0931A01A591A0931B01209232
:1064A0001C012092180120921901AF91FF91EF91E8
:1064B000089520921701409117014030E1F39DC0EB
:1064C000409116014030E1F708955FD0A2EBCA0F6A
:1064D000A2E0DA1FA881BA2FAF93A171BE7EB29558
:1064E000BA2BAF912092170140911701403041F42F
:1064F000409110014B3110F4A883F6CFB883F4CF4C
:10650000A8837BD042C03F933DED52D0209217012B
:10651000409114014470431749F0403021F40E9427
:106520002807342F03C00E944E07342F40911701D3
:10653000403061F4409110014B3120F448814F7795
:106540004883E6CF488140684883E2CF58815F772F
:1065500058833F910895D1E0C3EDCA0FD21D209218
:10656000170140911701403061F4409110014B3107
:1065700020F448814F774883F4CF488140684883AE
:10658000F0CF58815F7758830895AA2DBB2DDEE1A7
:10659000BD9FD1E0C8ECCA0FD21DC00DD11D08951A
:1065A000F6DF0F9302EBC00F02E0D01F0F910895AA
:1065B000D3E2BD9FD2E0C4E3CA0FD21DC00DD11DEE
:1065C0000895AA2DBB2DAA95B39525CDBF93B09163
:1065D0000C01B4FD0EC0BFEFB1B900001A99FECF97
:1065E00042B9B4E6BA95F1F72998B4E6BA95F1F74D
:1065F000299ABF9108954F9108954F9340912D018D
:1066000041FFF9CF4D7F40932D01FF93EF93DF932F
:10661000CF9340913E01403029F44091290147FF3A
:1066200013C02FC04F9347E4D8D04F914F93405D94
:10663000D4D04F91413009F45AC0423009F470C0AF
:10664000433009F48CC09EC044E50E94ED334AE01B
:106650000E94ED33C8ECD1E0FEE2EEE148814295C4
:10666000ADD04991ABD0EA95C9F74AE00E94ED332D
:10667000FA9599F7CF91DF91EF91FF914F914427D0
:10668000089545E40E94ED334091400194D04AE0E2
:106690000E94ED33C8ECD1E0F3E0E3E2488142959B
:1066A0008DD049918BD0EA95C9F74AE00E94ED332D
:1066B000FA9599F7E3E2F0912E01EF9FC00DD11DFD
:1066C000F0E1E3E248814F77429578D049914F77E6
:1066D00075D0EA95B9F74AE00E94ED33FA9589F74B
:1066E000CF91DF91EF91FF914F9144270895409111
:1066F000000161D0409101015ED04AE06ED0C8EC4B
:10670000D1E0F4E7E5E14881429558D0499156D06F
:10671000EA95C9F74AE00E94ED33FA9599F7E0CF80
:106720004091000148D04091010145D040910201C3
:1067300042D0409103013FD04AE04FD0C8ECD1E0B5
:10674000F4E5EEE14881429539D0499137D0EA9598
:10675000C9F74AE00E94ED33FA9599F7C1CF4AE0B4
:106760003CD0C8ECD1E0FAE3EAE24881429526D079
:10677000499124D0EA95C9F74AE00E94ED33FA9591
:1067800099F7AECF4091000116D04091010113D08E
:106790004AE023D0C8ECD1E0F0E4E0E14881429542
:1067A0000DD049910BD0EA95C9F74AE00E94ED332C
:1067B000FA9599F795CF4295469547704F70405D91
:1067C0004A3308F0495F0C94ED33BF93B2E0A03038
:1067D00009F0B064B4BDBF910895BF93B091250195
:1067E000B030E1F740932601BA95B0932501BF91EF
:1067F0000895BF93B0912701B030E1F7BA95B093F7
:106800002701B0912701B030E1F740912801BF91F5
:106810000895BF93B0912701B030E1F7BA95B093D6
:106820002701409116014D3E41F0B0912701B03053
:10683000C1F740912801BF9108954BE1BF910895A0
:10684000DF93CF93BF93AF93FF93EF93CEE0D7E067
:10685000E6ECF8E632D0EF91FF91FF93EF93CCE5B1
:10686000D4E0B0911401B2FD7E9616F026D001C09E
:106870001ED040911601A1E04D3E69F0A2E0413FDB
:1068800051F0A3E0423F39F0A4E0433F21F0A5E0FE
:10689000443F09F0E0CFB0911401B2FDAB5F4A2F45
:1068A000EF91FF91AF91BF91CF91DF910895BEE13C
:1068B000A191A993BA95E1F70895BEE1A591A99395
:1068C000BA95E1F708954E4E4E4E4E4EC0C0C0C030
:1068D000C0C08080808080802E2E2E2E2E2E6E6E48
:1068E0006E6E6E6EACE5B0910C01B3FDAFE5ACBD64
:1068F000ACE5A093B800A0E0B2FDA1E0A093B90080
:106900000895FF93EF930F93E0911E01A0911F0153
:10691000B0912001F09121010027E2FD0095E5FDF5
:106920000095A4FD0095F7FD0095001FEE1FAA1F1E
:10693000BB1FFF1FE0931E01A0931F01B093200116
:10694000F09321010F91EF91FF910895FF93EF9341
:10695000DF93CF93BF93AF934F935F936F937F93E7
:106960004F925F926F927F922F9320913E014090C1
:106970004601509049016090480170904B01509140
:10698000470160914A01A22FA370E52F660FEE0F19
:10699000A33031F0660FEE0FA23011F0660FEE0F4C
:1069A000F62FA0914C01A13071F4E20147D0803064
:1069B00011F08FE133C0E30141D0803011F080E26B
:1069C0002DC065D02BC0A23091F4E20137D08030C9
:1069D00011F08FE123C0E30140D0803011F082E15B
:1069E0001DC0ACE3BDE06A0E7B1E75D017C0A3309E
:1069F00011F085E113C0A52DA33010F082E10EC087
:106A0000ACE3BDE04A0E5B1EF20151916191E301DE
:106A100015D0803011F080E201C067D02F917F90B7
:106A20006F905F904F907F916F915F914F91AF9179
:106A3000BF91CF91DF91EF91FF910895CE0F10F4A8
:106A40008FE10895A0914401CA17D0F7DF0FC0F37A
:106A5000B0914501DB17A0F70895659FC00DD11DCA
:106A60002296D33008F082E10895A22F5091470179
:106A700060914A01E52F660FEE0FA33031F0660FEB
:106A8000EE0FA23011F0660FEE0FF62F0895571497
:106A900078F0D20134D0E0E8FBE064D0D3012FD00D
:106AA000E0E8FBE08CD0539473946A9591F70895D5
:106AB000560E760E5A947A94D20121D0E0E8FBE08B
:106AC00051D0D3011CD0E0E8FBE079D05A947A94FD
:106AD0006A9591F70895F30151936193D2010FD014
:106AE00041D053946A95D1F70895F2015191619183
:106AF000D30105D064D073946A95D1F708956F934C
:106B0000C8ECD1E0213011F465E103C0253069F40F
:106B100060E1B69FC00DD11D6A2F6695669566959A
:106B2000C60FD21D4A2F6F910895223069F46EE18D
:106B3000B69FC00DD11D6A2F66956695C60FD21DF2
:106B40004A2F440F6F9108956AE2B69FC00DD11D80
:106B50006A2F66956695C60FD21D4A2F440F440FC3
:106B60006F9108957F936F93BF93AF93652F742FA9
:106B7000777049F4A991A1936A95E1F7AF91BF911C
:106B80006F917F910895B0E8713019F0B6957A95BC
:106B9000FBCF7727A991AB9F703019F0A291A02964
:106BA000A193119273957617A9F7A991AB9FA29122
:106BB000A029A193AF91BF916F917F9108957F9389
:106BC0006F93BF93AF93652F742F777049F4A191A2
:106BD000A9936A95E1F7AF91BF916F917F91089565
:106BE0000F931F930FEF11E0000F110F7A95E1F74C
:106BF000652F7881009570230095A191A19F072AA8
:106C00000992712D6A95C9F768816023672B699392
:106C10000F911F91AF91BF916F917F910895BF9395
:106C2000AF934F939927A42F0E94E82D0E94632EC3
:106C30004F91AF91BF910895AF93BF93EF93FF939F
:106C40005F936F930F931F932F9310E020E0FAE868
:106C5000EE27509147015F7760914A016F77049169
:106C6000059FA12DE0950491E095069FB12DA117F8
:106C700029F4B21719F4E39591F724C01A2F2B2F9A
:106C8000A0914601B0914901A10FB20F0E941E30A0
:106C9000A0914601B0914901A10FB21B0E941E3084
:106CA000A0914601B0914901A11BB21B0E941E3068
:106CB000A0914601B0914901A11BB20F0E941E3064
:106CC000E39569F62F911F910F916F915F91FF915D
:106CD000EF91DF91AF910895AF93BF93EF93FF933F
:106CE0005F936F930F931F932F933F932FEFFAE8C8
:106CF000EE27509147015F7760914A016F770491C9
:106D0000059FA12DE0950491E095069FB12DB21746
:106D100021F4E395A1F73F91D5CF1A2F2B2FA09106
:106D20004601B09149013A2FB21BA11B310F0E94BD
:106D30001E30B20FB20F0E941E30B21BB21BA395C1
:106D40003A17A8F7E395D9F63F91BCCFFF91EF91A1
:106D5000EE0FFF1F5BD03197F695E7953196EF93D5
:106D6000FF93C8E7D1E040912C014F93FF93EF933D
:106D700061D00E94F22F0B092050524553532045F9
:106D80004E5445522000EF91FF914F9140932C01BA
:106D900090DB4A3EE9F794DB0E94F7190895FF91D2
:106DA000EF91EE0FFF1F32D03197F695E7953196B0
:106DB000EF93FF93C8E7D1E040912C014F93FF93ED
:106DC000EF9338D00E94F22F0B08202859296573C1
:106DD000202F20284E296F200000EF91FF914F9126
:106DE00040932C0166DB493761F0493551F04E364E
:106DF00019F04E3409F0F6CF63DB0E94F7194427EF
:106E000008955EDB0E94F71941E00895C8E7D1E0DC
:106E1000459146954F93477049934F9142954770DE
:106E2000499358E145914993403011F05A95D1F773
:106E300029920895FF93EF9392E020922A01A9915D
:106E4000B991B295B077A770AB0FAA0FA0932C01A0
:106E5000DF93CF930E94D119C2E0D8E0EBE1FCE0D0
:106E60000E945D31A3E0B9E00E940B30CF91DF9129
:106E700058E14991403051F0DF93CF935F930E94E6
:106E8000642E5F91CF91DF915A9599F740912C0133
:106E9000429540932C01EF91FF910895FF93EF935A
:106EA000DF93CF93BF93AF93C0914601D091490137
:106EB0000A8119810E3118F4173108F41AD0A09103
:106EC0004801B0914B01C0914601D0914901B9836D
:106ED000AA83AE3138F4B73128F43DD073707130E5
:106EE00009F076D0AF91BF91CF91DF91EF91FF91F3
:106EF0000895C0914601D09149010A8119812C81E0
:106F00003B81239F310F2596C00DD11DC00DD11D92
:106F1000412FE8ECF1E05EE1549FE00DF11DE00F40
:106F2000F21D522F699161935A95E1F743954317EA
:106F300081F7412FEAE7F4E05EE1549FE00DF11D97
:106F4000E00FF21D522F699161935A95E1F7439535
:106F5000431781F70895C0914601D09149010A81F4
:106F600019812C813B81239F310F2596C00DD11DA6
:106F7000C00DD11D7727412FE8ECF1E05EE1549F71
:106F8000E00DF11DE00FF21D522F619169936F70BA
:106F900009F071E05A95C9F74395431769F7E091F5
:106FA0004601F09149014081742B7083412FEAE73B
:106FB000F4E05EE1549FE00DF11DE00FF21D522F51
:106FC000619169935A95E1F74395431781F70895C5
:106FD000C0914601D09149010A8119812C813B81E0
:106FE000310F2596412FE8ECF1E05EE1549FE00D72
:106FF000F11DE00FF21D522F699161935A95E1F74F
:107000004395431781F7412FEAE7F4E05EE1549F8F
:10701000E00DF11DE00FF21D522F6991660F28F46B
:107020006E70462E6081607F642961935A95A9F73E
:107030004395431749F70895AF93BF93CF93DF93D9
:107040004F935F936F937F934F9270912C01437096
:10705000E1F4A6E0B2E0C4E2D2E0422C07D0A8EB13
:10706000B4E0C6EDD4E0472E01D061C062E15AE140
:1070700049914D935A95E1F7149624966A95B9F77C
:107080005AE14D925A95E9F708954130C9F4ACE3BD
:10709000B4E0CBE3D4E0422C07D0AEEEB6E0CDEEC8
:1070A000D6E0472E01D043C063E159E14A914E93A7
:1070B0005A95E1F74E92149725976A95B1F708957E
:1070C0004230E1F4ACE3B4E0CEE1D4E0422C07D0AE
:1070D000AEEEB6E0C0EDD6E0472E01D028C062E1AA
:1070E0005AE14A914E935A95E1F7149724976A957D
:1070F000B9F75AE14E925A95E9F70895A6E0B2E041
:10710000C7E0D2E0422C07D0A8EBB4E0C9EBD4E052
:10711000472E01D00CC063E159E149914D935A9536
:10712000E1F74D92259614966A95B1F708954F9020
:107130007F916F915F914F91DF91CF91BF91AF910F
:1071400008954F935F937F9364DB4B3111F481E09B
:1071500015C04130C9F74DDB642F4BDB40956417F8
:1071600011F088E20BC070E8552743DB540F4993B8
:107170007A95D9F73EDB451729F488277F915F91EF
:107180004F91089589E2FACF4F935F937F9341E047
:1071900024DB462F22DB409520DB70E85527499100
:1071A000540F1BDB7A95D9F7452F17DB7F915F9141
:1071B0004F9108955E984CE54093B80044E84093A1
:1071C000BC0044E94093BC00089544EA0EC05093CB
:1071D000BB0044E80AC044EC08D05091BB000895BD
:1071E00044E803D05091BB0008954093BC00409107
:1071F000BC0047FFFCCF6091B900687F0895E5DFD0
:10720000683089F4572F550F5E70506AE0DF68319F
:1072100051F45B2FDCDF683231F45A2FD8DF68324B
:1072200011F4882708958FE0CCCFCFDF6031D9F7F4
:10723000572F550F5E70516ACADF6034A1F7882757
:107240000895DDDF803049F4F0DF803031F4C8DFAD
:10725000683519F411968827B4CF8FE0B2CF5F93C9
:10726000CEDF5F91803031F4B2DF683219F41196CD
:107270008827A7CF8FE0A5CFA8DF6830A9F4572FC4
:107280005770550F5169A3DF603471F4A4DF603586
:1072900059F4A52FA5DF683539F4BB27550FAA1F70
:1072A00008F4B09588278DCF8FE08BCF8827D83012
:1072B00020F080E34F914F914FEF0895F7DFF99958
:1072C000FECFD2BDC1BDF89A40B521960895EEDF3C
:1072D000F999FECFD2BDC1BDF89A40B4441611F45D
:1072E0002196089554E040BDF894FA9AF99A78945A
:1072F000F999FECFF89A40B4441511F421960895F7
:10730000839580635A9579F70895AF93D7DF4193BA
:10731000AA95E1F7AF910895AF934191D8DFAA956F
:10732000E1F7AF9108954EBD4DB547FFFDCF4EB586
:10733000089588272C9847EDF6DF4427F4DF2C9A30
:107340004C7B4432B1F34C31A1F38827443A19F015
:107350004C3909F081E108958827EBDF803021F076
:1073600040E040939C1008954C3911F448E0F9CF67
:1073700040E1F7CFF1DF403009F40895440F440FA6
:10738000440F440F4A950895AA0FBB1F4B2FCBDF24
:107390004A2FC9DF422DC7DFB695A79508958030E3
:1073A00059F44F93C6DF803031F42C9845E5BBDFAC
:1073B000EBDF2C9ABEDF4F910895803059F44F9344
:1073C000B8DF803031F42C9843E5ADDFDDDF2C9A57
:1073D000B0DF4F910895803051F44F93AADF803091
:1073E00029F42C9846E89FDFCFDF2C9A4F9108951F
:1073F0001196B0939D10A0939E101197ECCF7F93A0
:10740000772710D07F9108957F9371E00BD0D42F10
:1074100072E008D0C42F7F9108957F9373E002D06B
:107420007F9108958030B9F484DF8030A1F42C98E6
:1074300042ED79DFAA0FBB1FA3954B2F74DF4A2FB4
:1074400072DF472F70DFB695A7956DDF6CDF6BDFBE
:107450006ADF69DF2C9A08958030D1F46ADF8030CA
:10746000B9F42C9842ED5FDFAA0FBB1F4B2F5BDFF7
:107470004A2F59DF472F440F56DFB695A79553DFA4
:1074800052DF51DF50DF4FDFD42F4DDFC42F2C9A56
:1074900008957F9370E010D07F9108957F9371E0FD
:1074A0004D2F0AD072E04C2FBDDF7F9108957F935E
:1074B00073E0B8DF7F9108958030A1F44F9339DFF6
:1074C0004F91803079F42C984F9347E82CDF442774
:1074D0002ADF41E028DF472F26DF4F914F9323DF3C
:1074E0002C9A4F910895803091F423DF8030D1F7AA
:1074F0002C984F9347E817DF442715DF40E013DF50
:10750000472F11DF4F914F930EDF2C9A4F91089523
:107510008030D1F4DF93CF934F935F930ADF8030B5
:1075200079F42C9847E8FFDE4427FDDE4427FBDE94
:1075300040E0F9DE55274991F6DE5A95E1F72C9A9D
:107540005F914F91CF91DF9108958030B1F44F93C7
:107550005F93EFDE803079F42C9847E8E4DE44272F
:10756000E2DE4427E0DE40E0DEDE55274FEFDBDEE3
:107570005A95E1F72C9A5F914F9108958030E1F48C
:10758000DF93CF934F935F93D4DE803089F42C98B0
:1075900046EDC9DE4427C7DE4427C5DE40E0C3DE32
:1075A0004427C1DE5527BFDE49935A95E1F72C9A4F
:1075B0005F914F91CF91DF910895BF93AF93DF9388
:1075C000CF934F935F937F93C7DE403041F47F9119
:1075D0005F914F91CF91DF91AF91BF910895B5DF4A
:1075E0004FE057DF442763DFAA27BB27F4DE11965D
:1075F0004DEFCA2FCF70C13009F44CEF4ADF44275A
:1076000056DFCC27DD274ADFE6DE1196A03019F4DD
:1076100045EE0E94642E40919C10B41749F7D7CFD5
:10762000BF93AF93DF93CF934F935F937F9394DE9A
:10763000403091F47F915F914F91CF91DF91AF9165
:10764000BF910895B42FAA271197E7DEC42FBB2757
:10765000AA27E3DE4C1731F4A2DEDFDE439527DFF5
:10766000BADEE8CF1196D9DE4C17E1F7F5CFDF93FC
:10767000CF934F9394DE4DEFCA2FCF70C13009F4F2
:107680004CEF07DFC1DE219609DF5FDFA4DE4F91FB
:10769000CF91DF910895FF93DF93CF93BF93AF9383
:1076A000AA27BB27ED0158DE4030A1F0F42FA7DE5A
:1076B0004C3F41F04D3F31F04B3A21F04F3018F044
:1076C000403908F421961196BF1789F74427DF1730
:1076D00009F441E0AF91BF91CF91DF91FF910895FF
:1076E0000F93BF93AF934F93AA27BB27ED01FD01E3
:1076F00033DE403099F0042F82DE4D3F49F4DF93B2
:10770000CF9382DE4D2FCF91DF914F3F21F0219615
:107710004C3F09F431961196B01771F74F91AF9124
:10772000BF910F910895FF93EF93DF93CF934F9302
:107730002F9312DE4030A9F0AA27BB2760DE242F4A
:10774000B0919D10A0919E1040910801B41710F0C7
:10775000A2E0BB27FD0153DE4D3F51F455DED217A9
:1077600038F42F914F91CF91DF91EF91FF910895D0
:10777000159640919C10B41709F4BB27BF1759F711
:10778000AE1749F7AA27BB270ADE39DE4F3F31F093
:10779000405F242F7EDE1FDEDF01DDCFAFEFBFEFC6
:1077A000E0CFFF93EF93DF93CF93BF93AF934F93CC
:1077B0005F936F937F93D0DD403061F481E17F91DF
:1077C0006F915F914F91AF91BF91CF91DF91EF9109
:1077D000FF91089551D0B41710F08BE1F0CF0FDE78
:1077E0004C3F11F087E1EBCF40915A01403011F44A
:1077F0008BE1E5CF413810F08BE1E1CF71DFD03084
:1078000021F4C41710F488E1DACFC0E8DBE050E0DF
:107810006FEF69935A95E9F798DE1196B0939D1032
:10782000A0939E1040915A01C0E8DBE04F937BDFAC
:10783000B993A9934BEA2DDEDF93CF93E5DD219633
:107840002DDECF91DF91E9DD32DED2DDE9DE4F9131
:107850004A9561F711D0C0E8DBE05ADE40915C0147
:1078600018DEDF93CF93D0DD219618DECF91DF9124
:10787000D4DD1DDEB0DDA3CFA0915801A295BA2FB3
:10788000A07FBF7011960895BF93AF93DF93CF93FE
:107890004F935F937F937727EFDFB1DD4C3F69F024
:1078A000DBDDDF3F49F0BF93AF93DE01E0DEAF9158
:1078B000BF91B6DE7F5FA1F7DADE7F915F914F91D6
:1078C000CF91DF91AF91BF910895BF93AF93DF93B5
:1078D000CF934F935F937F932F93AA27BB2729DDE5
:1078E0008EDD242FC9DF8BDD4C3F51F489E12F91D0
:1078F0007F915F914F91CF91DF91AF91BF910895AB
:1079000070915A01703810F08BE1F1CFA5DDDF3FA7
:1079100011F48BE1ECCFDE01CCE3DDE040915C01C2
:10792000413009F4D395423009F4DE5FF1DDDF9395
:10793000CF936ADDD21759F02196B0DDCF91DF9158
:107940005EDDA7DD6ADDB3DD46DD6ADED0CF8FDE2A
:10795000EADE5ADD2196A2DDCF91DF914BEA99DD77
:107960005CDDA5DD38DDED0187DF19DD70915A01A1
:10797000770F4D2FB8DD73954C2FB5DD40DD89DDD8
:107980004CDD95DD28DDB3CFBF93AF93DF93CF936D
:107990004F935F937F9370DF32DD4C3F49F48EE16C
:1079A0007F915F914F91CF91DF91AF91BF910895FA
:1079B00070915A01703810F08BE1F2CF4DDDDF3F4E
:1079C00011F48BE1EDCFDE01EADCCCE3DDE04091A8
:1079D0005C01413009F4D395423009F4DE5FCEDD1D
:1079E000DFCF0004080D11161A1F23282C3035395B
:1079F0003D42464A4F53575B5F64686C7074787CB5
:107A00007F83878B8F92969A9DA1A4A7ABAEB1B5C9
:107A1000B8BBBEC1C4C6C9CCCFD1D4D6D9DBDDDF9B
:107A2000E2E4E6E8E9EBEDEEF0F2F3F4F6F7F8F96C
:107A3000FAFBFCFCFDFEFEFFFFFFFFFFFFFF000067
:107A400000CCC000333000FFF000000CCCCCCCCC1C
:107A5000333CCCFFFCCC000333CCC333333333FF94
:107A6000F333000FFFCCCFFF333FFFFFFFFFA5A590
:107A7000A506FF60000000000000000000000000FC
:107A800000000000000000000000000000000000F6
:107A900000000EAE000004E000AAE800EE4E000078
:107AA00000444040AA000066FF666842C4A248A0A5
:107AB0000000004400004888404222400A4A000476
:107AC000E40000048000E000000040224880EAAAB0
:107AD000E04C44E0E2E8E0E2E2E0AAE220E8E2E0B2
:107AE000E8EAE0E24880EAEAE0EAE2E004040004CE
:107AF00004802484200E0E00842480C268E400EEFA
:107B0000E04AAEA0CACAC0688860CAAAC0E8C8E095
:107B1000E8C88068EA60AAEAA0E444E0E22A60AC2F
:107B20008CA08888E0AEAAA0CAAAA04AAA40EAE827
:107B3000804AAA60EAECA068E2C0E44440AAAAE055
:107B4000AAAA40AAAEA0AA4AA0AA4440E248E06479
:107B5000446004A400C444C04A00000000E04400A3
:107B6000004AAEA0CACAC0688860CAAAC0E8C8E015
:107B7000E8C88068EA60AAEAA0E444E0E22A60ACCF
:107B80008CA08888E0AEAAA0CAAAA04AAA40EAE8C7
:107B9000804AAA60EAECA068E2C0E44440AAAAE0F5
:107BA000AAAA40AAAEA0AA4AA0AA4440E248E02459
:0E7BB000C4204444448464808842208CEC80CD
:1086000000F900F5F3F1F2FC00FAF8F6F4EB5E0085
:10861000F7000000007131000000797361773200CB
:108620000063786465343300002076667472350028
:10863000006E6268677A360000006D6A7537380030
:10864000002C6B696F303900002E2D6C00707E009D
:1086500000000000002700000000EA2B00230000BB
:10866000003C00000000EC00003100343700000046
:10867000302C32353638ED00FB2B332D2A390000F3
:1086800000F900F5F3F1F2FC00FAF8F6F4EB000063
:10869000F70000000051210000005953415722000B
:1086A00000435844452440000020564654522500BB
:1086B000004E4248475A260000004D4A552F2800D8
:1086C000003B4B494F3D2900003A5F4C00503F00B2
:1086D00000000000006000000000EA2A00270000FF
:1086E000003E00000000EC000031003437000000C4
:1086F00030E932353638ED00FB2B332D2A390000B6
:108700000000000000000000000000000000000069
:108710000000000000000000000000000000000059
:108720000000000000000000000000000000000049
:1087300000000000000000C000000000000000C1B8
:10874000000000000000000000002F0000000000FA
:1087500000000000000000000000EA000000C2006D
:10876000000000000000000000E100E2E000000066
:10877000E8E9E500E3E4ED00FB2BE72D2AE6000045
:1087800000000000000000000000000000000000E9
:108790000000000000400000000000000000000099
:1087A00000000000000000000000000000000000C9
:1087B000000000000000000000000000007B5B00E3
:1087C00000000000007D5D000000000000007E0051
:1087D00000000000000000000000005C000000003D
:1087E000007C00000000000000E100E2E00000006A
:1087F000EFEEE500E3E4ED00FB2BE72D2AE60000B9
:1088000000F900F5F3F1F2FC00FAF8F6F4EB5E0083
:10881000F70000000071310000007A7361773200C8
:108820000063786465343300002076667472350026
:10883000006E62686779360000006D6A753738002F
:10884000002C6B696F303900002E2F6C3B702D00AF
:10885000000027005B3D00000000EA5D007E000094
:10886000000000000000EC00003100343700000080
:10887000302C32353638ED00FB2B332D2A390000F1
:1088800000F900F5F3F1F2FC00FAF8F6F4EB000061
:10889000F70000000051210000005A5341574000EA
:1088A00000435844452423000020564654522500D6
:1088B000004E424847595E0000004D4A55262A00A6
:1088C000003C4B494F292800003E3F4C3A505F0086
:1088D000000022007B2B00000000EA7D007C0000ED
:1088E000000000000000EC00003100343700000000
:1088F00030E932353638ED00FB2B332D2A390000B4
:108900000000000000000000000000000000000067
:108910000000000000000000000000000000000057
:108920000000000000000000000000000000000047
:1089300000000000000000C000000000000000C1B6
:10894000000000000000000000002F0000000000F8
:1089500000000000000000000000EA000000C2006B
:10896000000000000000000000E100E2E000000064
:10897000E8E9E500E3E4ED00FB2BE72D2AE6000043
:1089800000000000000000000000000000000000E7
:1089900000000000000000000000000000000000D7
:1089A00000000000000000000000000000000000C7
:1089B00000000000000000000000000000000000B7
:1089C00000000000000000000000000000000000A7
:1089D0000000000000000000000000000000000097
:1089E000000000000000000000E100E2E0000000E4
:1089F000E8E9E500E3E4ED00FB2BE72D2AE60000C3
:108A0000FFFFFFFFFFFFFFFFFFFFFFFEFEFEFEFE7B
:108A1000FEFEFDFDFDFDFDFCFCFCFCFBFBFBFBFA93
:108A2000FAFAF9F9F9F8F8F8F7F7F6F6F6F5F5F4D1
:108A3000F4F3F3F2F2F2F1F0F0EFEFEEEEEDEDEC35
:108A4000EBEBEAEAE9E8E8E7E6E6E5E4E4E3E2E1BD
:108A5000E1E0DFDEDEDDDCDBDADAD9D8D7D6D5D46B
:108A6000D4D3D2D1D0CFCECDCCCBCAC9C9C8C7C63A
:108A7000C5C4C3C2C1BFBEBDBCBBBAB9B8B7B6B529
:108A8000B4B2B1B0AFAEADACAAA9A8A7A6A5A3A237
:108A9000A1A09E9D9C9B99989796949392918F8E5E
:108AA0008D8B8A898786858382817F7E7D7B7A789C
:108AB0007776747371706F6D6C6A696766656362EF
:108AC000605F5D5C5A595756545351504E4D4B4A56
:108AD0004847454442413F3E3C3B393836353332C6
:108AE000302E2D2B2A2827252422201F1D1C1A1941
:108AF00017161412110F0E0C0B09070604030100C0
:108B00000C11161A1E2225282B2D2F313233333407
:108B100034343434343434343535363738393B3CF6
:108B20003E40434547494B4D4F5152535454545482
:108B3000545351504E4C4A4745423F3D3A383634E3
:108B40003231302F2E2E2E2F303132333536383A07
:108B50003C3E4042444647494A4B4D4E4E4F505092
:108B60005050505050504F4E4D4C4B494846434149
:108B70003E3B37332F2B27221D18130D0802FDF81B
:108B8000F3EEE9E5E1DDDAD7D4D2D0CECDCCCCCB53
:108B9000CBCBCBCBCBCBCBCBCACAC9C8C7C6C4C344
:108BA000C1BFBCBAB8B6B4B2B0AEADACABABABAB98
:108BB000ABACAEAFB1B3B5B8BABDC0C2C5C7C9CB17
:108BC000CDCECFD0D1D1D1D0CFCECDCCCAC9C7C5D3
:108BD000C3C1BFBDBBB9B8B6B5B4B2B1B1B0AFAF28
:108BE000AFAFAFAFAFAFB0B1B2B3B4B6B7B9BCBE51
:108BF000C1C4C8CCD0D4D8DDE2E7ECF2F7FD02075F
:108C0000000A141D272F383F464B505457595959C5
:108C1000585654504C48433E39332E2925201C19B0
:108C200016141211111112131517191C1F222527C2
:108C30002A2C2E303132323232312F2D2B28252260
:108C40001F1C191613110F0D0C0B0A0A0A0B0C0E20
:108C500010121416181A1C1E1F2020201F1E1C196B
:108C600016120D0803FDF7F0EAE3DDD6D1CBC6C23C
:108C7000BFBDBBBABBBCBEC2C6CBD1D7DFE6EFF728
:108C80000008101920282E34393D41434445444200
:108C9000403D39342E29221C150F0802FCF7F2ED55
:108CA000E9E6E3E1E0DFDFDFE0E1E3E5E7E9EBED83
:108CB000EFF1F3F4F5F5F5F4F3F2F0EEECE9E6E3B9
:108CC000E0DDDAD7D4D2D0CECDCDCDCDCECFD1D37D
:108CD000D5D8DADDE0E3E6E8EAECEDEEEEEEEDEB3A
:108CE000E9E6E3DFDAD6D1CCC6C1BCB7B3AFABA9F6
:108CF000A7A6A6A6A8ABAFB4B9C0C7D0D8E2EBF57B
:108D000080675342352B221C16120E0C09070605EC
:108D1000040000000000000000000000000000004F
:108D20000000000000000000000000000000000043
:108D30000000000000000000000000000000000033
:108D40000000000000000000000000000000000023
:108D50000000000000000000000000000000000013
:108D60000000000000000000000000000000000003
:108D700000000000000000000000000000000000F3
:108D8000890091009A00A300AD00B700C200CE0098
:108D9000DA00E700F4000301120123013401460167
:108DA0005A016E0184019B01B301CD01E901060264
:108DB0002502450268028C02B302DC020803360376
:108DC00067039B03D2030C0449048B04D0041905E8
:108DD0006705B90510066C06CE063507A307170808
:108DE000930815099F09320ACD0A720B200CD80C82
:108DF0009C0D6B0E460F2F1025112A123F13641481
:108E0000F894A0E02A2EA1E03A2EA0E1AEBFAFEF89
:108E1000ADBFB0E0A0E0AA95F1F7BA95D9F7AAEBFB
:108E2000A4B9AFEFA5B9A0E8A7B9A0E0A8B9A0EF91
:108E3000AAB9AFEFABB9A6B1AF71A09329014B9915
:108E40005DC0B2ECB0938000B9E1B0938100F4E072
:108E5000A2FFF4E0F0938700FEEFA2FFF6EFF0939D
:108E6000860020928900FAE5F0938800A2E0A093A2
:108E70006F00A0E4A4BDA1E0A5BDA1E3A7BD209221
:108E8000C000A0E1A093C100A6E6A093C200E0EA62
:108E9000FFE87ED0A2E2B591B993AA95E1F705B7B4
:108EA000036005BF0E7F05BF7894A8EC68D0B09131
:108EB000C600B83719F0AA95C9F720C0E0ECFFE862
:108EC00067D045E140D0C8ECD1E020D046E03BD0AF
:108ED000E0E0F0E0CCE3DFE019D046E034D0CCEBCA
:108EE000DFE014D0FE3820F40E946B79329678943B
:108EF00046E029D0AEEDB1E01BD0ECCFF89405B739
:108F0000016005BF0C7F05BF0C94000028D04430E1
:108F100039F446E018D0B0912501B030E1F7EECF3A
:108F200050E81DD01CD01BD049935A95E1F717C0CB
:108F30004F2F429501D04F2F4F70405D4A3308F0BC
:108F4000495F4D930895BF93B0912501B030E1F78B
:108F500040932601BA95B0932501BF910895BF9320
:108F6000B0912701B030E1F7BA95B0932701B091E5
:108F70002701B030E1F740912801BF910895AF93E8
:108F8000A82DA73EE9F3A82DA73EE9F7AF910895D4
:108F9000C8ECD1E0A2E2B591B993AA95E1F70895A2
:108FA0004156522D436869704261736963322028CB
:108FB0004631313D557064617465205379732920C1
:108FC000426F6F746C6F61646572204572726F726C
:108FD000202845534320746F206578697429202028
:0E90000020202020202020202020202078006A
:0E9C000020202020202020202020202078005E
:0EA80000202020202020202020202020780052
:0EB40000202020202020202020202020780046
:0EC0000020202020202020202020202078003A
:0ECC000020202020202020202020202078002E
:0ED80000202020202020202020202020780022
:0EE40000202020202020202020202020780016
:10F000000C94004700000000000000000000000019
:10F0100000000000000000000000000000000000F0
:10F0200000000000000000000000000000000000E0
:10F03000000000000C941C784F935F936F93FF9334
:10F04000EF93DF93CF93BF93AF930F921F92FFB7CE
:10F05000FF93C8E0D1E0B9A5B7FF5C98B7FD5C9A13
:10F060004B99BE7F4B9BB160B9A7830C921CE9A161
:10F07000F92DF03029F4F82DFA3010F1F63EF8F0C1
:10F08000FCE0E2FFFDEE8F1639F45E98E3FF17C057
:10F09000B2E8B093800013C0F1E1E2FFF3EF8F1606
:10F0A00039F45E9AE3FF0BC0B2ECB093800007C066
:10F0B000F9E3E2FFF7E08F1611F4882499242CC0BD
:10F0C000A0918400AA3FE0F3AB3F00F0AC3F00F01A
:10F0D000AD3F00F0AE3F00F0A8ECB1E0F6EFF80D68
:10F0E000C0E2ED91549140E060E848B9ED9156FDE1
:10F0F00066B90000000055FD66B9049054FD66B97C
:10F10000CA95000053FD66B90000000052FD66B9C3
:10F11000502D59F7000028B814D0E091C600E6370A
:10F1200011F40C947E47FF91FFBF1F900F90AF9199
:10F13000BF91CF91DF91EF91FF916F915F914F91CF
:10F140001895A0913101E0912701E03091F0EF3F57
:10F1500021F4A0FD0EC0EEE30CC0EA95F5EFB491EA
:10F16000B5FF07C0B0912801B695A0FBB7F9B093E1
:10F170002801E0932701E0912501E03091F0EF3F75
:10F1800019F4E8E4AF770DC0EA95F5EFB491B4FF58
:10F1900008C0B0912601B0FB0894B795A7F9B093C9
:10F1A0002601E0932501A09331010895A09131013A
:10F1B000E0912701E03091F0EF3F21F4A0FD0EC077
:10F1C000ECE70CC0EA95F5EFB491B7FF07C0B0913A
:10F1D0002801B695A0FBB7F9B0932801E093270169
:10F1E000E0912501E030E9F2EF3F19F4E0E9AF7773
:10F1F000D8CFEA95F5EFB491B6FFD3CFB091260101
:10F20000B0FB0894B795A7F9B0932601CACF4091F7
:10F210000C01C8EFD7E00E9467390895C8EFD7E026
:10F220000E945E3940930C010895FF93EF93DF93A2
:10F23000CF93AF93F4D0E0933401F0933501AF91C5
:10F24000CF91DF91EF91FF910895E0E0F0E9C0E008
:10F25000DCE0A42FA03021F0EC0FFD1FAA95FACF1F
:10F260000895E0913401F0913501A0E2A99FE00DED
:10F27000F11DB096C0EAD1E0A0E2B591B993AA958C
:10F28000E1F7BFEFB993089547B740FDFDCFB7BF92
:10F29000E89547B740FDFDCF089547B746FF08956D
:10F2A000B1E1F2DFFACFF8944E2F407E19F4B3E0CB
:10F2B000EBDFF3DFA0E109901990B1E0E5DF3296D2
:10F2C000AA95C9F7E03009F008953297B5E0DCDF80
:10F2D000E4DF32960895F8944F93BF93AF93B3E071
:10F2E000D3DFDBDF3297CCE3DFE0A0E83296099092
:10F2F0001990B1E0C9DFAA95C9F7B5E0C5DFCDDF48
:10F30000AF91BF914F910895E0913401F091350193
:10F31000B097ACE0B591B993AA95E1F7A091290116
:10F32000A7FD0895A6EAB2E0CA0FDB1FACE0B091DA
:10F330002C01B993AA95E9F70895E0E0F0E9A0E07F
:10F34000BCE0492F403029F3EA0FFB1F4A95FACF62
:10F35000F89463D0C0EAD1E0A3EDB1E05CE04D9158
:10F3600049935A95E1F742E4499353E140E2B99356
:10F370005A95E9F7A09797DF9927B3E2B99FA4E3DD
:10F38000B2E0A00DB11DC8E7D1E050E24D91499324
:10F390005A95E1F7299250E24A91403219F42882B5
:10F3A0005A95D1F70E943918C0EAD1E07CDF9395D5
:10F3B0009F3519F77894089530D0A3EDB1E05CE063
:10F3C00045914D935A95E1F77496992750E2A0EA3A
:10F3D000B1E045914D935A95E1F7A8E7B1E040E2DD
:10F3E00053E24D935A95E9F7FF93EF939F930E9451
:10F3F00023199F91EF91FF91C8E7D1E0B3E2B99F44
:10F40000A1E3B2E0A00DB11D53E249914D935A958D
:10F41000E1F793959F35D1F6089540913D01AF9363
:10F42000BF93E0E0F0E947704295A0ECA49FE00DA7
:10F43000F11DBF91AF910895CCE3DFE04CE050E2C5
:10F4400059934A95E9F75FEF599343E150E2599395
:10F450004A95E9F740EF5FEF59934A95E9F7DDDF09
:10F460003ADF3296CCE3DFE040E25FEF59934A9512
:10F47000E9F74BE04F932FDF32964F914A95D1F742
:10F4800078940895472F4770CADFFF93EF93C5DF45
:10F49000AF91BF914CE04F93CCE3DFE040E055915A
:10F4A00059934A95E1F7FF93EF93FD0114DF3296EC
:10F4B000DF01EF91FF914F914A9569F77894089594
:10F50000010101010101210101010101013181011B
:10F510000100003100010101010131C101010101BE
:10F520003101010101010131C1010101013101017B
:10F530000101010131C101010101110101010101BB
:10F540000111C1010101010101010101010101C11B
:10F55000010101010101010101000101C1010101DC
:10F56000010101010101010001C1010101010100CD
:10F57000010101010101410001010101010101003D
:10F58000000000400000000000000000000000003B
:10F59000000000000000000000000000000000006B
:10F5A000000000000000000000000000000000005B
:10F5B000000000000000000000000000000000004B
:10F5C000000000000000000000000000000000003B
:10F5D000000000000000000000000000000000002B
:10F5E000100000000000000000000000000000000B
:10F5F00020000000000000000000000000000000EB
:10F60000009010800090108000901080009010807A
:10F61000FC28288004C0145028282800000000007E
:10F6200000000000000000000000000000000000DA
:10F6300000000000000000000000000000000000CA
:10F6400000000000000000000000000000000000BA
:10F6500000000000000000000000000000000000AA
:10F66000000000000000000000000000000000009A
:10F67000000000000000000000000000000000008A
:10F6800028C004C00000000000000000000000804E
:10F69000C0A0888400000000000000002088FCB4A6
:10F6A0000028000008A08080000004C028800024FA
:10F6B00000008000000044288000C004C41800003E
:10F6C000000000000000000000000000C004000076
:10F6D0008090808008A084408080C8A400004C8472
:10F6E0000000000000000000C00480800080282886
:10F6F000280000002828002828282800002CE8904E
:10F700000090108000901080009010800090108079
:10F710007C444480A8A814504844440024000000BD
:10F7200000183C3C185028280C3000000000000055
:10F73000241824400C401440242400000C003024E1
:10F7400024244424444040246424106460646424D9
:10F7500044244424406464646464404800481800BD
:10F76000300060000400140060180C6028000000E5
:10F7700000000000300000000000000C18306000A5
:10F7800028A004C0808044283C3C3C000044A88061
:10F79000C0A08884000000000000008040847C58E5
:10F7A000182800001090808004C004C028FC287C29
:10F7B00000440C00000044EC8000C004C42400009D
:10F7C000000000000000000000008080C004000075
:10F7D0008088A41010908440C004C8A400008C80CD
:10F7E000287C008080004084FCF4C0040000244891
:10F7F000280000002828002828282800002CE8C01D
:10F800000090108000901080009010800090108078
:10F81000FC44448080801450444444283C00000050
:10F8200000183C3C20546C181818181800000004EC
:10F830006428640C14603064646428281800186418
:10F84000646464646460606464180C6C605864642C
:10F8500064646464186464646464046000183C0054
:10F860001800600004003400600000601800000010
:10F870000000000030000000000000181818601898
:10F88000449008A0C4C4806C0000001C1844A880E8
:10F89000C0A0888400000000000080804084FCB488
:10F8A0002428282820888080A4A00C60448044401C
:10F8B00000440C40844444800000C0046C24004494
:10F8C00000000000000000000000C004C004481058
:10F8D0008084BCB020888820D834C8A440848C8020
:10F8E0002C7C00C4C444C004E094C0040080208880
:10F8F000280000002828002828282800002CE8A03C
:10F900000090108000901080009010800090108077
:10F910007C808080808010908480804424186424BF
:10F9200000183C40780C7830300C7C180000000C3B
:10F93000681804183C44600C6464282830400C04A7
:10F94000046464606460606064180C78607C546473
:10F9500064646460186464643C640C60301864001F
:10F960000C2444242C2430207428146C185C742437
:10F970004824742448646464646440181818300C83
:10F9800044881090C4BC446C24246434286C6C807B
:10F99000C0A08884000000000080808080807CEC13
:10F9A000404444442088408490A00C6044FC286477
:10F9B00000440C40844444280000C0046C240080AF
:10F9C00000000000000000000000C004C00418187F
:10F9D0008080BC1040848820E82CC8A480804C849F
:10F9E000EC2400C4EC44C004E094C00400802088EF
:10F9F000280000002828002828282800002CE8E4F7
:10FA00000090108000901080009010800090108076
:10FA1000FC808080B098109080ECEC44003C6464E2
:10FA20000018003C24183000300C2440004000181E
:10FA30007C180C0C6C044418242000006000040C9A
:10FA40002C6444606444447040180C50607C7C64B6
:10FA50004464442418646464183C18607C180000F2
:10FA6000000464606864486454180C78187C54641A
:10FA70006C6C5460306464643C640C30180C188006
:10FA800080841090C4F8806C04646440406C6C8086
:10FA9000C0A0888400000000808080808080FCB44A
:10FAA0001880442840844084808418308080282432
:10FAB00000440C40844444440000C00428241880BE
:10FAC00000000000000000000000C004C00440244A
:10FAD000A4B0BC4080808080E82CC8A488104084FA
:10FAE000E42400C4EC44F434E094C0048080208812
:10FAF000288020882088808020888020882CE8F03A
:10FB00000000000090909090101010108080808075
:10FB10007C8080801090B098408080440040646475
:10FB2000001800401C307800300C7C182800003091
:10FB300054181804400464186404282830400C1831
:10FB40007C4064606460606464180C78606468641D
:10FB5000607C780418643C7C3C1830600C18000011
:10FB6000002064606440306464180C50187C646445
:10FB70006C6C602430646464182C181818180C0C11
:10FB800080842088C4C444C420646430286C6C80A1
:10FB9000C0A08884000000008080808080807CEC91
:10FBA00018008044408440848080301880FC801895
:10FBB00000448040844444440000C004280024449D
:10FBC00000000000000000000000C004C004244049
:10FBD000BCD0A41084404084E82CC8A44C8480800D
:10FBE000482400C4EC44EC7CE094C004808020886D
:10FBF000288020882088808020888020882CE82801
:10FC00000000000090909090101010108080808074
:10FC1000FC8080801090808084C4A8440000643CF4
:10FC20000000003C44686C00181818181800286080
:10FC3000641830640C646430640C281818001800D0
:10FC40007C6464646460606464186C6C60646464A4
:10FC500060686C6418643C7C641860600018000084
:10FC6000006464646460302064180C781864646410
:10FC7000482460043C683C7C3C0830181818041880
:10FC800044882088C4C4808064646818186C6C80C0
:10FC9000C0A0888400000080808080808080FCB4C8
:10FCA000400080804084208880843018DC80284098
:10FCB00000446040844444280000C0046C0024C414
:10FCC00000000000000000000000C004C00418187C
:10FCD000BCB0808084402088E44CC4C44C848080C4
:10FCE000282400C4EC44F87CFCF4C00480002828DC
:10FCF000280028280000280028282820882CE83000
:10FD00000000000090909090101010108080808073
:10FD10007C4480441450808044EC442800004458C3
:10FD20000018003C18082C000C300000300028009F
:10FD3000242440240C242430242800300C003018C3
:10FD4000246444244440602464242864406464247B
:10FD5000602C64241824182464184048004800408B
:10FD6000002044242424300464246C6C246464241F
:10FD7000600C6044182C183C6404400C18300400DB
:10FD8000449040848080442820242C0000A8448093
:10FD9000C0A08884000080808080808040847C585F
:10FDA000240080288080208890A0600CDCFC44180F
:10FDB00000446040844444EC0000C0046C00240013
:10FDC00000000000000000000000C004C004104853
:10FDD000BCB0808080801090D094C0048C8040841F
:10FDE000284000C4C444F44CC004C0048000282847
:10FDF000280028280000280028282820882CE830FF
:10FE00000000000090909090101010108080808072
:10FE1000FC4480441450A8A84080440000006000C6
:10FE200000000000000000000000000000000000D2
:10FE300000000000000000000000000000000000C2
:10FE400000000000000000000000000000000000B2
:10FE500000000000000000000000000000000000A2
:10FE60000000000000000024000028000000000046
:10FE700060080000000000000024000000000000F6
:10FE800028A08080000000000000000000A844803E
:10FE9000C0A0888400808080808080804084FCECCA
:10FEA0001800444480801090A4A0C004DC806C3C06
:10FEB00000446000004400800080C004C4002400AE
:10FEC00000000000000000000000C004808000006E
:10FED000A4B08080844008A0C8A480808C800000EA
:10FEE000444000808000F47C4084C0040000282846
:10FEF000280028280000280028282824482CE8006A
:10FF00000000000090909090101010108080808071
:10FF10007C2880281450109080EC28000000C0003D
:10FF200000000000000000000000000000000000D1
:10FF300000000000000000000000000000000000C1
:10FF400000000000000000000000000000000000B1
:10FF500000000000000000000000000000000000A1
:10FF60000000000000000000000000000000000091
:10FF70000000000000000000000000000000000081
:10FF800028C0808000000000000000000000008009
:10FF9000C0A08884808080808080808020887C5879
:10FFA00000004480808008A004C0C0048CFCA858D5
:10FFB00000006000004400280080C004C40000006D
:10FFC00000000000000000000000C004000000006D
:10FFD0008080000084400000C8A400004824000085
:10FFE000000000000000C0040000C00480002828B9
:10FFF000280028280000280028282828282CE80085
:00000001FF
